:10142400758400852ED2852FD37584018530D285AD
:1014340031D3E4F52FF52E30005730064E855B820C
:10144400855A83E0F52FA3E0F52EA385825B85837F
:101454005AE55B655D700CE55A655C7006755B006A
:10146400755A02855982855883E533F0A3E532F035
:10147400A3858259858358E559655D7014E55865DF
:101484005C700E755900755802800685322E8533BE
:101494002F30010CE52E2534F52EE52F3535F52FAB
:1014A400300210E53F8527F0A4252EF52EE5F03512
:1014B4002FF52F300310E50A852AF0A4252EF52EEA
:1014C400E5F0352FF52F300410E5118529F0A4251A
:1014D4002EF52EE5F0352FF52FE4F531F5303009F2
:1014E4005730054E855B82855A83E0F531A3E0F5DC
:1014F40030A385825B85835AE55B655D700CE55A94
:10150400655C7006755B00755A028559828558833F
:10151400E535F0A3E534F0A3858259858358E55970
:10152400655D7014E558655C700E75590075580258
:10153400800685343085353130080CE5302532F5A8
:1015440030E5313533F531300A10E53F8527F0A415
:101554002530F530E5F03531F531E531C3952C40D2
:0315640003852CD0
:1015670031300B10E50A852AF0A42530F530E5F077
:101577003531F531300C10E5118529F0A42530F50A
:1015870030E5F03531F531300D10E5188528F0A438
:101597002530F530E5F03531F531E531C3952D408E
:1015A70003852D31229016053015031215C230160A
:1015B700031215D23018031215F522E50B2509F58C
:1015C7000BE50C3508F50C93F50A22E512250EF507
:1015D70012E513350DF51393C313F8E5142510F52C
:1015E70014E515350FF51593C31328F51122E519E1
:1015F7002517F519E51A3516F51A93F518227F827E
:1016070085888C8F9295989B9EA1A4A7AAADB0B30D
:10161700B6B9BBBEC1C3C6C9CBCED0D3D5D7D9DC2B
:10162700DEE0E2E4E6E7E9EBEDEEF0F1F2F4F5F601
:10163700F7F8F9FAFBFCFCFDFDFEFEFEFEFEFEFEE2
:10164700FEFEFEFDFDFCFCFBFAFAF9F8F7F6F4F3F3
:10165700F2F0EFEDECEAE8E7E5E3E1DFDDDBD8D632
:10166700D4D1CFCDCAC8C5C2C0BDBAB7B4B2AFAC6A
:10167700A9A6A3A09D9A9794908D8A8784817E7A44
:101687007774716E6B6865625F5C595653504D4A4B
:101697004744423F3C393734322F2D2A282624210C
:1016A7001F1D1B1918161412110F0E0C0B0A080711
:1016B7000605040403020201010000000000000007
:1016C70000000001010202030405060708090A0BCE
:1016D7000D0E1011131516181A1C1E202224272967
:1016E7002B2E303335383A3D404245484B4E515406
:1016F70056595C606366696C6F7275787B7FFEFE16
:10170700FEFEFDFCFCFBFAF8F7F6F4F3F1EFEDEB68
:10171700E9E7E4E2DFDCDAD7D4D0CDCAC6C3BFBC81
:10172700B8B4B0ACA8A39F9B96928D89847F7A7535
:10173700706B66615C57514C47413C37312C262111
:101747001B16100B050000050B10161C21272C3249
:10175700373D42484D53585D62686D72777C81858D
:101767008A8F94989DA1A5AAAEB2B6BABEC1C5C8C4
:10177700CCCFD2D5D8DBDEE1E3E6E8EBEDEFF1F253
:10178700F4F6F7F8F9FBFBFCFDFEFEFEFEFE000C8F
:101797001926333F4C5864707B86919CA6AFB8C11D
:1017A700C9D1D8DEE4EAEFF3F6F9FCFDFEFEFEFD53
:1017B700FCFAF7F4F0EBE6E0DAD4CCC5BCB4ABA1A5
:0E17C700978D83786D61554A3D3125180C00D1
:101E6000D2F4C2F5C2F675840F85F0C812254A7403
:101E700003121EAF12253E7403121EAF122521124B
:101E800025217403121EAF1225217402121EAF12F7
:101E900025217428121F1B7406121F1B740E121F9B
:101EA0001B7401121F1B12253E7480121F1B22C0BF
:101EB00000A2E092F3A2E192F2A2E292F1A2E392F6
:101EC000F0D2F475840F85F0C8C2F47830D8FE855E
:101ED000F0C87830D8FED00022C00075840FA2E48C
:101EE00092F3A2E592F2A2E692F1A2E792F0D2F486
:101EF00085F0C8C2F47830D8FE85F0C87830D8FEB6
:101F0000D00022EF75840FD2F5C2F685F0C8121EFC
:101F1000D9122521121EAF1225212275840FC2F578
:101F2000C2F685F0C8121ED9122521121EAF122545
:101F30002122EF14A2E492E6C2E4D2E7121F1B2290
:101F4000740F121F1B22740D121F1B227F01121F00
:101F50003278107F20121F03D8F9227F11121F320E
:101F600078107F20121F03D8F9227F01121F3278C8
:101F7000207F20121F03D8F922C0077F018004C0F0
:101F8000077F11121F32D007C082C083C007EF75D0
:101F9000F010901FAA1225627810E493FF121F031D
:091FA000A3D8F7D007D083D0824A
:101FA9002220202020202020202020202020202026
:101FB9002057414954494E4720464F522052494ED5
:101FC900472054454C434F20414E535745524544B1
:101FD90020205741495420464F5220444953434FEA
:101FE9002020205445535420204641494C45442043
:101FF9002020205445535420205041535345442018
:10200900202020454550524F4D20544553542020FF
:1020190020204155582052454C415920544553548C
:102029002020205055534820544F2054414C4B20D8
:102039002054455354203320434841522F5355428D
:102049002054455354204649584544205354524935
:102059004E544553542056415249422053545249F3
:102069004E464143544F52592044454641554C54DC
:102079002050524F4752414D4D494E47204D4F44F4
:102089004553494D504C45582052455045415445BA
:10209900522020205245434F5244494E4720202088
:0120A9002016
:102AC60032C28D32758400C2CF32C0E0C083C0826C
:102AD600C0D0C000C0F0C2CFB21A201A23121424EC
:102AE600151BE51B7009751B0A7584017588AF15E2
:102AF6001CE51C7009751C607584027588AF801111
:102B06001215AC1536E5367008753604758400D294
:102B16008B758400D2ECD0F0D000D0D0D082D08398
:102B2600D0E032C2CF32C0E0C0D0C007C000C08300
:102B3600C08212455575888FD082D083D000D007C9
:102B4600D0D0D0E032C0E0C0D0C000C083C082C0C8
:102B56008420121375840F30DF27E5E8540FF54003
:102B6600D2127541C8801A1541E5417006E540D27A
:102B7600E7F54075840F20DF08C212D211D22AD29F
:102B86002D20141475840F30F828E5E854F0C4F5A8
:102B960042D2147543C8801A1543E5437006E542D0
:102BA600D2E7F54275840F20F808C214D213D22951
:102BB600D21C12459A151DE51D702A751D0A12456F
:102BC600C1151EE51E701E751E0A124614151FE558
:102BD6001F7012751F061246151526E52670067516
:102BE600260A12461ED084C28DD082D083D000D051
:102BF600D0D0E0323220100DD21085BF3585BE34DC
:0A2C060075BB01800BC21085BF33BF
:102C100085BE3275BB00C2ED32C0E0C0D0E544B421
:102C2000000A054485BE3F75BB07803DB4010A0517
:102C30004485BE3C75BB048030B4020A054485BEA1
:102C40003F75BB068023B4030A054485BE3D75BBB2
:102C5000048016B4040A054485BE3F75BB0580098F
:102C600075440085BE3E75BB04C2EDD0D0D0E032C5
:103E590044313233343536373839302A23414243F5
:103E6900202020205354414E444259202020202014
:103E7900524144494F204F524947494E41544520E8
:103E890054454C434F204F524947494E41544520D0
:103E990020202046554E4354494F4E2031202020A2
:103EA90020202046554E4354494F4E203220202091
:103EB90020202046554E4354494F4E203320202080
:103EC90020202046554E4354494F4E20342020206F
:103ED90020202046554E4354494F4E20352020205E
:103EE90020202046554E4354494F4E20362020204D
:103EF90020202046554E4354494F4E20372020203C
:103F090020202046554E4354494F4E20382020202A
:103F190020202046554E4354494F4E203920202019
:103F2900202052454345495645204D4F44452020C0
:103F3900205452414E534D4954204D4F4445202061
:103F4900202045204C4541442044454C41592020DE
:103F5900205741495420464F52204D204C45414459
:103F690020524144494F2045204C454144202020BE
:1046270012694D124AE875840F1200A412694112EB
:10463700625F12629812655C125A0F20A503120E70
:10464700DA9000A5E4F020A432302915C229E5420A
:10465700540FFFEF903E5993FF90008CEFF01251EB
:104667005E302AE2C22AE540540FFFEF903E59938D
:10467700FF90008BEFF01251D080CB9000A5E0FFA8
:10468700EF12435846B00046B50146BA0246BF038B
:1046970046C40446C90546CF0646D50746DB084645
:1046A700E10946E70A0000464D125D968098123FE1
:1046B700798093125819808E1265898089122C701F
:1046C7008084122FB102464D124B7E02464D126076
:1046D700FE02464D125C7302464D12675402464D68
:0A46E700124D1702464D02464D2207
:105D960012673A1269351269411268331264D112D8
:105DA600655C125E69126A039000ACE4F09000B183
:105DB600E4F09000A6E4F09000EEE4F09000EDE44C
:105DC600F07BFF7A3E7969126445121F5B753832A3
:075DD6009000A5E004F0229B
:103F7900E538600302408B124C9512558D302B0B9E
:103F890012662CC22B9000A5E4F022301F0B12629E
:103F9900D1C21F9000A5E4F0221267EB50409000B7
:103FA900E1E0FF9000A7EFF09000EBE0FFEFB40233
:103FB9000312692F9000ECE0FFEFB4020312693B92
:103FC9009000B1E4F07BFF7A3E79891264457BFF6A
:103FD9007A3F79491264769000A57402F02212673B
:103FE900FDEF604D9000EAE0FFEF64017043126855
:103FF900439000E2E0FF9000A8EFF09000EBE0FFB3
:10400900EFB4020312692F9000ECE0FFEFB4020352
:1040190012693B9000B1E4F07BFF7A3E7979126432
:10402900457BFF7A3F79591264769000A57406F0B2
:1040390022126971404C9000EAE0FFEF640270427D
:104049001268439000E2E0FF9000A8EFF09000EBC7
:10405900E0FFEFB4020312692F9000ECE0FFEFB428
:10406900020312693B9000B1E4F07BFF7A3F796962
:104079001264457BFF7A3F79591264769000A574E2
:0340890006F0221C
:10581900121B759000A7E0FFEF702D1268439000EE
:10582900EBE0FFEFB4020312692F9000ECE0FFEF09
:10583900B4020312693B75370A7BFF7A3F79291253
:1058490064769000A57403F0124C95302B0B126608
:105859002CC22B9000A5E4F022301F0A1262D1C29B
:075869001F9000A5E4F022EE
:10658900121B75E53770231269EB1269B812673A65
:106599009000D8E0FF9000A3EFF09000EDE4F090B8
:0B65A90000EEE4F09000A57405F02265
:102C700020A60312545D1269B5121B751217D512E6
:102C8000531E12558D12408C124C959000EEE0FFB1
:102C9000EF603F12673A1268339000EBE0FFEF6499
:102CA0000160099000EBE0FFEFB402031269359078
:102CB00000ECE0FFEF640160099000ECE0FFEFB48E
:102CC00002031269419000EF740AF09000A57409A4
:102CD000F0229000DBE0FFEF705C9000A6E0FFEFD9
:102CE000602B900098E0FFEF70239000A6E4F09036
:102CF0000099E4F09000DEE0FF9000D9E0FEEE2FB6
:102D0000FF9000A1EFF09000A5740AF022900098C7
:102D1000E0FFEF702190009CE0FFEF70199000DE63
:102D2000E0FF9000D9E0FEEE2FFF9000A1EFF090C1
:102D300000A5740AF0229000DBE0FFEFB4012190BF
:102D40000098E0FFEF70199000DEE0FF9000D9E0FE
:102D5000FEEE2FFF9000A1EFF09000A5740AF02284
:102D60009000DBE0FFEFB4022190009CE0FFEF70E9
:102D7000199000DEE0FF9000D9E0FEEE2FFF9000FA
:102D8000A1EFF09000A5740AF0229000DBE0FFEFC5
:102D9000D3940240219000B1E0FFEF70199000DE63
:102DA000E0FF9000D9E0FEEE2FFF9000A1EFF09041
:102DB00000A5740AF022302B2012673A12693512EE
:102DC000694112683312662CC22B1269D61269DC73
:102DD0001269B89000A5E4F022301F1D12673A1264
:102DE00069351269411269D61269DC1269B812623A
:102DF000D1C21F9000A5E4F0221267EB40189000AA
:102E0000DEE0FF9000D9E0FEEE2FFF9000A1EFF092
:072E10009000A57408F022F8
:102FB10020A60312545D12687212667A121B7512F2
:102FC10017D51269DC1269D612531E12558D1240A3
:102FD1008C124C959000EEE0FFEF603F12673A12C1
:102FE10068339000EBE0FFEF640160099000EBE0D3
:102FF100FFEFB402031269359000ECE0FFEF6401CA
:1030010060099000ECE0FFEFB40203126941900007
:10301100EF740AF09000A57409F0229000DBE0FF44
:10302100EF701A900098E0FFEF700E90009CE0FFA7
:10303100EF600A1267FDEF7004125E24229000DB3C
:10304100E0FFEFB4010C900098E0FFEF6004125E26
:1030510024229000DBE0FFEFB4021290009CE0FF1D
:10306100EF600A1267FDEF7004125E24229000DB0C
:10307100E0FFEFB4030C9000B1E0FFEF6004125EDB
:1030810024229000DBE0FFEFB4040C9000B1E0FFDC
:10309100EF6004125E2422302B2012673A12693548
:1030A1001269411268331269EE12662C1269D61246
:1030B10069EEC22B9000A5E4F022301F1D12673A81
:1030C1001269351269411269D61269B81269EE1294
:1030D10062D1C21F9000A5E4F0221267EB404012BA
:1030E100683312673A9000EBE0FFEF6401600990EA
:1030F10000EBE0FFEFB402031269359000ECE0FF52
:10310100EF640160099000ECE0FFEFB40203126983
:10311100411269D61269DC1269B89000A5E4F02267
:104B7E009000EAE0FFEFB4011312558D1267FDEFBE
:104B8E00600A9000E2E0FF9000A8EFF09000EAE0EB
:104B9E00FFEFB4020F126971400A9000E2E0FF903D
:104BAE0000A8EFF09000A8E0FFEF70299000E2E07F
:104BBE00FFEF60211268339000EBE0FFEFB40203C9
:104BCE001269359000ECE0FFEFB4020312694190D8
:104BDE0000A5E4F0221267EB500975370A9000A584
:104BEE007407F0124C95302B0B12662CC22B9000D2
:104BFE00A5E4F022301F0A1262D1C21F9000A5E474
:024C0E00F02292
:1060FE001267EB400375370AE537701275370A7B66
:10610E00FF7A3F79291264769000A57403F0124C41
:10611E0095302B0B12662CC22B9000A5E4F022308A
:0D612E001F0A1262D1C21F9000A5E4F022EA
:105C73009000A1E0FFEF704012683312673A900082
:105C8300EBE0FFEF640160099000EBE0FFEFB4028B
:105C9300031269359000ECE0FFEF640160099000A6
:105CA300ECE0FFEFB402031269411269D61269DC1A
:095CB3001269B89000A5E4F0228A
:106754009000EFE0FFEF700E1269D61269DC126947
:07676400B89000A5E4F0224B
:104D17009000A1E0FFEF700412640E221269B51231
:104D27001B751217D512408C124C95302B0B12663F
:104D37002CC22B9000A5E4F022301F0B1262D1C2C7
:104D47001F9000A5E4F0229000EEE0FFEF603E1216
:104D5700673A1268339000EBE0FFEF640160099057
:104D670000EBE0FFEFB402031269359000ECE0FFBF
:104D7700EF640160099000ECE0FFEFB402031269F1
:0E4D8700419000EF740AF09000A57409F0222C
:105E24001269EE126A06125DDD1269B89000E8E0AC
:105E3400FFEF60069000AE7401F01267209000EB53
:105E4400E0FFEFB4010312692F9000ECE0FFEFB420
:105E5400010312693B7BFF7A3F7939126476900023
:055E6400A57404F0220A
:10640E007BFF7A3F79291264761269B81269EB1212
:10641E00673A9000EBE0FFEFB4010312693590008C
:10642E00ECE0FFEFB401031269419000A57405F092
:01643E00223B
:106833009000E0E0FFEF60041269472212694D22E5
:106843009000E0E0FFEF600412694D2212694722D5
:1067EB009000DFE0FFEF6006126977B32222126997
:0267FB00772203
:10418D00900091E0FF703B9000CAE060159000CB6D
:10419D00E0FEE53ED39E40249000CCE090009302DB
:1041AD0042459000CBE0FEE53EC39E500F9000CC03
:1041BD00E0900093F09000917403F022E49000944D
:1041CD00F022EF640170249000CBE024FBFFE53E6C
:1041DD00D39F406C900093E060030242889000945E
:1041ED0004F09000CDE0900092804D900091E0FFA2
:1041FD00B402179000CBE024FBFEE53ED39E4002B7
:10420D00805F900092E070738066EF64037033906E
:10421D0000CBE02405FFE433FEC3E53E9FEE648052
:10422D00F8748098501A900093E0704F90009404A9
:10423D00F09000CDE0900092F0900091E004F0221B
:10424D008034900091E06404702C9000CBE0240544
:10425D00FFE433FEC3E53E9FEE6480F87480985012
:10426D00099000CDE0900092F022900092E0700B4A
:0C427D00900094F08001E4900091F02289
:10552C00900091E0700E12695350559000CCE090B1
:10553C000093801E900091E0B40122126953501A1E
:10554C00900093E0701790009404F09000CDE090E0
:10555C000092F0900091E004F022E4801F90009102
:10556C00E0B4021C12695350099000CDE0900092F7
:10557C00F022900092E07008900094F0900091F06E
:01558C0022FC
:0D6872009000C9E0600302552C12418D22F8
:10408C00900095E0FF703B9000CEE060159000CF63
:10409C00E0FEE53DD39E40249000D0E090009702D6
:1040AC00414C9000CFE0FEE53DC39E500F9000D0F8
:1040BC00E0900097F09000957403F022E490009843
:1040CC00F022EF640170259000CFE024FBFFE53D6A
:1040DC00D39F4074900097E0701290009804F09079
:1040EC0000A6F09000D1E09000968054900095E0EE
:1040FC00B402179000CFE024FBFFE53DD39F4002B4
:10410C008064900096E07002806B900095E0FF64F4
:10411C000370379000CFE02405FDE433FCE53DC38C
:10412C009DEC6480F8748098501E900097E0701A93
:10413C0090009804F09000A6F09000D1E0900096CA
:10414C00F0900095E004F0228031EF6404702C9024
:10415C0000CFE02405FFE433FEC3E53D9FEE648011
:10416C00F874809850099000D1E0900096F022905D
:10417C000096E07006900098F08001E4900095F0B5
:01418C002210
:10531E00900099E0701912695F500E9000D4E090E1
:10532E00009BF0900099E004F0E490009CF0229035
:10533E000099E0B4012212695F501A90009BE07050
:10534E001790009C04F09000D5E090009AF0900029
:10535E0099E004F022E4801F900099E0B4021C1240
:10536E00695F50099000D5E090009AF02290009A63
:0C537E00E0700890009CF0900099F02274
:10558D0090009DE0700E12695950559000D2E09038
:10559D00009F801E90009DE0B40122126959501A9F
:1055AD0090009FE070179000A004F09000D3E09061
:1055BD00009EF090009DE004F022E4801F90009D7D
:1055CD00E0B4021C12695950099000D3E090009E7E
:1055DD00F02290009EE070089000A0F090009DF0E9
:0155ED00229B
:1067FD009000D7E060069000A0E0FF22900094E0AA
:02680D00FF2268
:10667A009000D8E0FF601D90009CE070069000A09A
:10668A00E060069000A3EFF0229000A3E07005906E
:05669A00009004F02255
:1050EB0054564F582020434F53202053454E534581
:1050FB00004F4E2020202020202020202020202068
:10510B0020004F4646202020202020202020202039
:10511B00202000191823A01296203D129623A012CE
:10512B009627631488203D148823A01488276316C0
:10513B00B8203D16B823A016B827631918203D19BF
:10514B0018276312962B8C14882B8C16B82B8C1962
:03515B00182B8C82
:104AE80012699112698E126953E433F54F12699471
:104AF800E433F54F126997E433F54F12699AE433BA
:104B0800F54F12699DE433F54F1269A0E433F54F70
:104B18001269A3E433F54F1269A6E433F54F12691D
:104B2800A9E433F54F126965E433F54F1269ACE433
:104B380033F54F126971E433F54F1269AF1269B258
:104B48001269BB1269BE1269C11269C41269C7121F
:104B580069CA1269CD1269D01269DF1269E2126955
:104B6800E51269E81269F11269F41269F71269FA33
:064B78001269FD026A0053
:06692F0075840FD2FC226A
:0669350075840FC2FC2274
:06693B0075840FD2B722A3
:0669410075840FC2B722AD
:0669470075840FD2FE2250
:06694D0075840FC2FE225A
:1067200075840FD2FD9000EBE0B4010312692F9045
:0A67300000ECE0B4010312693B2203
:10673A0075840FC2FD9000EBE0B401031269359035
:0A674A0000ECE0B4010312694122E3
:03698E00C293228F
:03699100D293227C
:0669530075840FA2FA2278
:03699400A2A0229C
:03699700A2A12298
:03699A00A2A22294
:03699D00A2A32290
:0369A000A2A4228C
:0369A300A2A52288
:0369A600A2A62284
:0369A900A2A72280
:0669590075840FA2F92273
:06695F0075840FA2DD2289
:0669650075840FA2DE2282
:0369AC00A2922292
:06696B0075840FA2DA2280
:0669710075840FA2DB2279
:0669770075840FA2DC2272
:06697D0075840FA2D82270
:0669830075840FA2D92269
:0369AF00D20822E9
:0369B200C20822F6
:0369B500D20922E2
:0369B800C20922EF
:0369BB00D20A22DB
:0369BE00C20A22E8
:0369C100D20222DD
:0369C400C20222EA
:0369C700D20B22CE
:0369CA00C20B22DB
:0369CD00D20C22C7
:0369D000C20C22D4
:0369D300D20D22C0
:0369D600C20D22CD
:0369D900D21822AF
:0369DC00C21822BC
:0369DF00D20E22B3
:0369E200C20E22C0
:0369E500D20F22AC
:0369E800C20F22B9
:0369EB00D20022B5
:0369EE00C20022C2
:0369F100D20122AE
:0369F400C20122BB
:0369F700D20322A6
:0369FA00C20322B3
:0369FD00D204229F
:036A0000C20422AB
:105DDD00E4FDFCED25E0FFEC33FE74002FF582743D
:105DED00023EF583E4F0A3F00DBD00010CBC0EE303
:105DFD00BDE0E07558027559007402F55AF55B90D7
:105E0D0000D9E075F0BEA4AEF02400F55DEE3402CD
:065E1D00F55CC200D20595
:015E2300225C
:036A0300C20522A7
:105E6900E4FDFCED25E0FFEC33FE74002FF58274B0
:105E7900023EF583E4F0A3F00DBD00010CBC0EE376
:105E8900BDE0E07558027559007402F55AF55B904A
:105E990000D9E075F0BEA4AEF02400F55DEE340241
:045EA900F55CD206CC
:015EAD0022D2
:036A0600C20622A3
:0B68AF0075081575095ED215D2032292
:0B68BA0075081575095ED215D20B227F
:07692100C215C203C20B22E4
:0B68C5009000BD12328CD216D20422CB
:0B68D0009000BE12328CD216D20C22B7
:0C328C00E0F529E4F512F513F514F51532
:10329800EF12435833932333822A32D03032E2314B
:1032A80032F432330633331834332A35333C363369
:1032B8004E3733603833713933A44133B54233C69E
:1032C8004333D744000033EF90511EE493F50D7457
:1032D8000193F50E9051200233E6905122E493F5C4
:1032E8000D740193F50E9051240233E6905126E4B3
:1032F80093F50D740193F50E9051280233E6905121
:103308002AE493F50D740193F50E90512C0233E6DF
:1033180090512EE493F50D740193F50E90513002FF
:1033280033E6905132E493F50D740193F50E905104
:10333800340233E6905136E493F50D740193F50E9B
:103348009051380233E690513AE493F50D740193A5
:10335800F50E90513C0233E690513EE493F50D741E
:103368000193F50E9051408075905142E493F50D0C
:10337800740193F50E9051448064905146E493F59E
:103388000D740193F50E905148805390514AE4937F
:10339800F50D740193F50E90514C804290514EE416
:1033A80093F50D740193F50E905150803190515260
:1033B800E493F50D740193F50E90515480209051CB
:1033C80056E493F50D740193F50E905158800F90C3
:1033D800515AE493F50D740193F50E90515CE49302
:0833E800F50F740193F51022AA
:07692800C216C20CC20422DA
:05698900C215C203224B
:0B68DB007508027509ABD215D20B2224
:0B68E60075081A7509ABD215D20B2201
:10545D0012531E12558D7BFF7A5079EB12644590D5
:10546D00009CE07BFF60067A5079FC80047A5179CC
:10547D000D1264767F17121F32AF3E1225A79000D2
:10548D006CE0FF121F0390006DE0FF121F039000F0
:10549D006EE0FF121F037F1C121F32AF3D1225A7B6
:1054AD0090006CE0FF121F0390006DE0FF121F03D0
:0854BD0090006EE0FF021F03E6
:10024D0020202020202020202020202020202020A1
:10025D002020202020202020202020202020202091
:10026D002054454C434F2050524F4752414D202072
:10027D0020524144494F2050524F4752414D20206A
:10028D002054574F20544F4E45204D4F444520206C
:10029D0020434F4D50552050524F4752414D202035
:1002AD00202041434345535320434F4445202020B4
:1002BD0044544D462054454C434F204C4556454CD7
:1002CD0044544D4620524144494F204C4556454CCF
:1002DD004245455020524144494F204C4556454CCE
:1002ED00424545502054454C434F204C4556454CB6
:1002FD0054454C434F20524144494F204C45564C98
:10030D00524144494F2054454C434F204C45564C87
:10031D00524144494F204C494D4954204C45564C6F
:10032D002045494120544F4E45204C4556454C20C3
:10033D004C4F57204755415244204C4556454C2073
:10034D0048494748204755415244204C4556454C55
:10035D00564F494345205241444930204C45564C57
:10036D00564F4943452054454C434F204C45564C20
:10037D0020434F53204F5220535155454C43482055
:10038D002020434F5320504F4C4152495459202067
:10039D00434F53205452494747455220564F4C54D2
:1003AD00434F5320414351554953542054494D45D2
:1003BD00434F532052454C454153452054494D45DB
:1003CD002053454E534520504F4C415249545920CE
:1003DD0053454E205452494747455220564F4C5491
:1003ED0053454E20414351554953542054494D4591
:1003FD0053454E2052454C454153452054494D459A
:10040D005220564F582041435155495354494F4E50
:10041D0020525820564F582052454C4541534520A7
:10042D005420564F582041435155495354494F4E2E
:10043D0020545820564F582052454C454153452085
:10044D00204F5045524154494E47204D4F44452071
:10045D0020564F58204F5220434152524945522069
:10046D002020564F58204143544956495459202075
:10047D00202054454C434F2044454C4159202020C9
:10048D002020524144494F2044454C4159202020C1
:10049D0053454E53452C20564F582C20544F4E4506
:1004AD0020204143434553532044454C415920207E
:1004BD00205455524E204F4E2044454C415920203A
:1004CD00205455524E204F46462044454C4159200C
:1004DD004449474954414C20494E20504F4C4152BC
:1004ED00434E544C2052454C415920504F4C415293
:1004FD002020452D44454C41592050425820202064
:10050D002020452D44454C41592052454320202063
:10051D00202052494E474F5554204D4F44452020E1
:10052D00414E535745522052494E47204E4D42524F
:10053D0020202052494E4720535041434520202032
:10054D00202052494E4720414E53574552202020DE
:10055D0052494E47205452414E534954494F4E53E0
:10056D0045494120544F4E4520454E41424C452072
:10057D0046554E4354494F4E20382053454C454324
:10058D00524144494F2053454C454320454E424C22
:10059D00204155582052454C4159204D4F4445203E
:1005AD002043542052454C4159204D4F4445202065
:1005BD00202020202020202020202020202020202E
:1005CD00202020202020202020202020313D454E9D
:1005DD002020202020202020202020524154494F2F
:1005ED002020202020202020202020303D434F534C
:1005FD002020202020202020202020313D504F532E
:10060D0020202020202020202020202031204D536C
:10061D0020202020202020202020203130204D534C
:10062D0020202020202020202020313030204D532C
:10063D002020202020202020202020202053454332
:10064D00202020202020202020202020204D494E19
:10065D002020202020202020202020204D4F4445E8
:10066D002020202020202020202020313D564F58B2
:10067D00202020202020202020202052494E47538A
:10068D0020202020202020202020204359434C458D
:10069D0020202020202020202020313D544F4E4569
:1006AD002020202020202020504F4C4152495459C9
:1006BD008201001102381500018201011103381564
:1006CD000001820102110438150001820103110598
:1006DD003815000178060411060119000082030A7D
:1006ED001107391500FF82030B1108391500FF8220
:1006FD00030C1109391500FF82030D110A3915007C
:10070D00FF82030E110B391500FF82030F110C39F7
:10071D001500FF820310110D391500FF8203111111
:10072D000E391500FF820312110F391500FF8203D8
:10073D00131110391500FF8203141111391500FF23
:10074D008203151112391500FF82011611133A1586
:10075D00000182011711143B1500018203181115B8
:10076D00391500FF82021911163C15006382021A19
:10077D0011173D15006382011B11183B15000182F5
:10078D00031C1119391500FF82021D111A3C1500A9
:10079D006382021E111B3D15006382021F111C3C5A
:1007AD00150063820220111D3E1500638202211186
:1007BD001E3C150063820222111F3E15006382014B
:1007CD00231120411500028201241121421500013F
:1007DD0082022511224015006382022611233D1548
:1007ED00002882022711243D150028820128112599
:1007FD004115000482022911263E150A6382022A40
:10080D0011273C15006382022B11283D15006382D0
:10081D00012C11294615000182012D112A461500C2
:10082D000182022E112B3D1501FF82022F112C3E4C
:10083D00150063820130112D3C150001820131112B
:10084D002E43150009820232112F3C1500638201DF
:10085D00331130411500018203341131441501FF6C
:10086D0082013511323815000182013611334515DB
:10087D00000182013711343715000282013811351C
:10088D004115000382013911364115000320202046
:10089D002020202020202020202020202082010127
:1008AD0011020C15000120202020202020202020C6
:1008BD0020202020202082010111020C1500012092
:1008CD0020202020202020202020202020202064D7
:1008DD0001001102091500012020202020202020D8
:1008ED0020202020202020200101010101010101F3
:1008FD0001000000000000000000000000000000EA
:10090D0000000000000000000000000000000000DA
:10091D0000000000000000000000000000000000CA
:10092D0000000000000000000000000000000000BA
:10093D0000000000000000000000000000000000AA
:10094D0000002020202020202020202020202020DA
:10095D002020010101010101010101000000000041
:10096D00000000000000000000000000000000007A
:10097D00000000000000000000000000000000006A
:10098D00000000000000000000000000000000005A
:10099D00000000000000000000000000000000004A
:1009AD0000000000000000000000000020202020BA
:1009BD0020202020202020202020202001010101A6
:1009CD000101010101000000000000000000000015
:1009DD00000000000000000000000000000000000A
:1009ED0000000000000000000000000000000000FA
:1009FD0000000000000000000000000000000000EA
:100A0D0000000000000000000000000000000000D9
:100A1D000000000000002020202020202020202089
:100A2D0020202020202082010011021E150001012E
:100A3D00010101313233343536FF323232FFFFFFDF
:100A4D00550CFF3232000180000A0080000A000AB6
:100A5D00000A0001002828001E140000012863016F
:100A6D000163000A01010102000000000000000006
:100A7D0044313233343536373839302A2341424305
:100A8D0044AAA3C1C2C3C4D7ABA8A92A23414243D8
:100A9D0036333036373036393437313937343437F9
:100AAD0037303739373832353835343838353931DC
:100ABD0035393438393734313030313033313037EE
:100ACD0031313031313431313831323331323731F6
:100ADD0033313133363134313134363135313135DD
:100AED0036313539313632313635313637313731B8
:100AFD0031373331373731373931383331383631A2
:100B0D003839313932313936313939323033323091
:100B1D003632313032313832323532323932333396
:100B2D003234313235303235343030363030373092
:100B3D003135303137303231303233303235303289
:100B4D00363033313033323033363034333034376E
:100B5D003035303035313035333035343036353061
:100B6D00373130373230373330373431313431314A
:100B7D003531313631323231323531333131333243
:100B8D00313334313431313433313435313532312F
:100B9D00353531353631363231363531373231370B
:100BAD003432303532313232313432323332323511
:100BBD0032323632343332343432343532343632F2
:100BCD0035313235323235353236313236333236E1
:100BDD0035323636323731323734333036333131D0
:100BED0033313533323533333133333233343333C9
:100BFD0034363335313335363336343336353337A2
:100C0D0031343131343132343133343233343331B0
:100C1D003433323434353434363435323435343487
:100C2D00353534363234363434363534363635306F
:100C3D00333530363531363532333532363533326C
:100C4D003534363536353630363631323632343651
:100C5D003237363331363332363534363632363640
:100C6D00343730333731323732333733313733323C
:100C7D0037333437343337353441424344454647AF
:100C8D0048494A4B4C4D4E4F50515253545556575F
:100C9D0058595A6162636465666768696A6B6C6D01
:100CAD006E6F707172737475767778797A303132C0
:100CBD0033343536373839607E21402324255E267E
:100CCD002A28295F2D2B3D7B7D5B5D7C3A3B3C3E8D
:100CDD002C2E3F2F202020202020202020202020BF
:100CED0020474C4F42414C202020202020204354AF
:100CFD0043535320434F444520202020202020449F
:100D0D00435320434F44452020202020204C545253
:100D1D0020524550454154455220202020535045E6
:100D2D004544204449414C494E47202020535045CD
:100D3D0045442043414C4C494E47202020205054DF
:100D4D0043204E554D424552202020202020564F05
:100D5D00494345204D455353414745532020564F58
:100D6D0049434520504C41594241434B2020204995
:100D7D004E56414C49442054595045202020204F77
:100D8D005554204F462052414E4745202020494C76
:100D9D004C4547414C2056414C554520204D55530F
:100DAD00542046494C4C204649454C44202020496E
:100DBD004C4C4547414C20434F4445202020444155
:100DCD00544120414343455054454420204C494E05
:100DDD0045204E554D4245523A2020202055534531
:100DED00522050524F4752414D4D494E4755534554
:100DFD00522049443A2020202020202020564F49BF
:100E0D004345205245434F5244494E472020494CBB
:100E1D004C4547414C20454E545259202020494CB9
:100E2D004C4547414C2047414E4720202020202053
:100E3D00434F4D504C455445442020202020474CD5
:100E4D004F42414C20454550524F4D2020202043CC
:100E5D005443535320454550524F4D2020202020C0
:100E6D0044435320454550524F4D202020202020F3
:100E7D004C545220454550524F4D2020202044497E
:100E8D00414C494E4720454550524F4D202043413E
:100E9D004C4C494E4720454550524F4D2020202067
:100EAD0050544320454550524F4D2020202052454F
:100EBD0050454154455220454550524F4D202049F3
:0D0ECD004E495449414C495A494E47202096
:1062D1009000A47464F0E4900000F030200B301FB3
:1062E10024125FBD12271A80F530210B301F1612C0
:1062F1005FFF12271A80F530220B301F0812291375
:0663010012271A80F522AC
:10271A009000A4E07012900000E0D394004009C237
:10272A0020C221C222C21F22900000E01243582870
:10273A003300283601283902283C03283F0428415F
:10274A0005284306284507284808284B0A284E0B1F
:10275A0028510F285410285714285A15285D19286B
:10276A00601A28631B28661E28691F286C23286F95
:10277A002428722828752928782D287B2E287E2F30
:10278A00288130288432288733288934288C3528B0
:10279A008F64289265289566289867289B6E289DDD
:1027AA006F289F7028E17128A17828A37928A57A33
:1027BA0028E17B28A78228A98328AB8428AD85280D
:1027CA00B08C28B38D28B58E28B78F28BA9628BD25
:1027DA009728BF9828C19928C4A028C7A128CAA2A7
:1027EA0028CCA328CFAA28D1AB28D4AC28D6AD2888
:1027FA00D9B428DCB528DFB628E1B728E3BE28E635
:10280A00BF28E9C028ECC128E1C228F2F028F5F176
:10281A0028F8F228FBFA28FEFB2901FC2904FD29E5
:10282A0007FE290AFF0000290D02680F0266E3026B
:10283A005EAE0265DE800480028000025C290231FD
:10284A00210263A70233F00258C602353E02591A22
:10285A0002368C02604102564E023BC4025AAE0254
:10286A0037DA025AFA023928025B46023A760265D8
:10287A0000026226025CBC125BDE0257658000021F
:10288A0052B0025F7A02596E025EF2026307025781
:10289A00BF80468032804B804080228045800780FE
:1028AA0026803F025B920246F1801C80350259BFA6
:1028BA00024D958008802B026080024863025241D3
:1028CA0080200247B18012024F888016023D0F0213
:1028DA004F0C0253F4800B800C025001025A5F0223
:1028EA0049B302613B02587002660502538A0268C4
:1028FA0053025709026A12026A13026A14024E123A
:09290A00026A15E4900000F022BD
:10680F00E4900002F09000A47464F0900000E004A3
:02681F00F02265
:1066E300121F4C121F5B7BFF7A0D79EA1264457F00
:0F66F30011121F32C226C223900000E004F022D1
:105EAE00302340900001E0FFC223BF2A079000007C
:105EBE00E004F022EF6423702A7F23121F03900068
:105ECE0002E004F0E0C394034013C220C221C222B8
:105EDE00C21FE4900000F01265B4021F6A90000029
:035EEE007402F04B
:015EF100228E
:1065DE007BFF7A0D79EA126445121F5B7F11121F41
:1065EE003212687FE490003CF07F2A121F03C2260D
:0765FE00900000E004F02210
:105C2900302346900001E0F55EC223E55E642A60F8
:105C390038AF5E1268635022AF5E121F0390003CBA
:105C4900E02403F582E43400F583E55EF090003C3E
:105C5900E004F0900000E004F0227BFF7A0E791A4C
:095C690012644590000074FAF089
:015C7200220F
:1031210020230302328B900001E0FFC223BF2A0754
:103131009000007403F022EF6423600302327C12DA
:103141001F03900004E064397077A3E06439707163
:10315100A3E06439706BD227900003E0FFB431081B
:10316100E4900036F00231EBEFB43208E49000371E
:10317100F00231FEEFB43302803E900003E0FFB471
:103181003408E4900038F002322CEFB43508E490B2
:103191000039F0023242EFB43608E490003AF0020E
:1031A1003258EFB437028010900003E0B438028047
:1031B10007900003E0B4390B7BFF7A0E792A0232C3
:1031C10082C227900003E0FFB43016A3E0B43011AF
:1031D100A3E0B4300CA3E0B43007900000740AF00F
:1031E10022EFB4310C1256AC5007900000740FF06E
:1031F10022900003E0B4320C1255EE50079000000B
:103201007414F022900003E0B43311A3E0B4300C45
:103211001266C250079000007419F022900003E07A
:10322100B4340FA3E0B4300A126782900000741E18
:10323100F022900003E0B4350FA3E0B4300A126726
:10324100979000007423F022900003E0B4360FA39E
:10325100E0B4300A1267AC9000007428F0229000AC
:1032610003E0B43716A3E0B43011A3E0B4300CA3EB
:10327100E0B43007900000742DF0227BFF7A0E79C4
:0A3281001A12644590000074FAF080
:01328B002220
:1063A70090003B740BF090003C7407F0E4900049B8
:1063B700F090004A743AF0E490004BF07BFF7A0CBF
:1063C70079EA1264451264707F1E121F3290000032
:0463D7007432F0220A
:1033F000125076D3900072E09434900071E0940003
:10340000400A12643F90000074FAF022900071E0CC
:10341000FEA3E0FF9006BD75F00912434CEE75F077
:1034200009A42583F583E493900040F09006BE75CF
:10343000F009EF12434CEE75F009A42583F583E4FF
:1034400093900041F0900071A3E09006BF75F009E1
:1034500012434CEE75F009A42583F583E4939000A4
:1034600042F09006C075F009EF12434CEE75F0097A
:10347000A42583F583E493900043F0900071A3E0CA
:103480009006C175F00912434CEE75F009A425832E
:10349000F583E493FD900044F09006C275F009EFC7
:1034A00012434CEE75F009A42583F583E493900054
:1034B00045F0900071A3E09006C375F00912434CEB
:1034C000EE75F009A42583F583E493900046F0900F
:1034D00006C475F009EF12434CEE75F009A425837C
:1034E000F583E493900047F0900071A3E09006C547
:1034F00075F00912434CEE75F009A42583F583E4B9
:1035000093900048F0ED6015900044E075F010A431
:10351000244DF9740235F0FA7BFF126445900045A2
:10352000E0FF601175F010A4244DF9740235F0FA33
:0E3530007BFF126476900040E0900000F022D5
:1058C60090003B7410F090003C7407F0900049740F
:1058D6003AF0E490004AF0900036E090004BF07BFE
:1058E600FF7A0C79FA1264451264707F0D121F322A
:1058F600900004E0FF121F03900005E0FF121F0353
:10590600900006E0FF121F037F1E121F3290000058
:045916007432F022D5
:10353E00125076D3900072E09400900071E09400E7
:10354E00400A12643F90000074FAF022900071E07D
:10355E00FEA3E0FF9008AA75F00912434CEE75F039
:10356E0009A42583F583E493900040F09008AB7591
:10357E00F009EF12434CEE75F009A42583F583E4B0
:10358E0093900041F0900071A3E09008AC75F009A3
:10359E0012434CEE75F009A42583F583E493900055
:1035AE0042F09008AD75F009EF12434CEE75F0093C
:1035BE00A42583F583E493900043F0900071A3E07B
:1035CE009008AE75F00912434CEE75F009A42583F0
:1035DE00F583E493FD900044F09008AF75F009EF89
:1035EE0012434CEE75F009A42583F583E493900005
:1035FE0045F0900071A3E09008B075F00912434CAD
:10360E00EE75F009A42583F583E493900046F090BF
:10361E0008B175F009EF12434CEE75F009A425833D
:10362E00F583E493900047F0900071A3E09008B208
:10363E0075F00912434CEE75F009A42583F583E469
:10364E0093900048F0ED6015900044E075F010A4E2
:10365E00249AF9740835F0FA7BFF12644590004500
:10366E00E0FF601175F010A4249AF9740835F0FA91
:0E367E007BFF126476900040E0900000F02286
:10591A0090003B7415F090003C7407F090004974B5
:10592A003AF0E490004AF0900037E090004BF07BA8
:10593A00FF7A0D790A1264451264707F0C121F32C5
:10594A00900004E0FF121F03900005E0FF121F03FE
:10595A00900006E0FF121F037F1E121F3290000004
:04596A007432F02281
:10368C00125076D3900072E09400900071E0940098
:10369C00400A12643F90000074FAF022900071E02E
:1036AC00FEA3E0FF9008C375F00912434CEE75F0D1
:1036BC0009A42583F583E493900040F09008C47529
:1036CC00F009EF12434CEE75F009A42583F583E461
:1036DC0093900041F0900071A3E09008C575F0093B
:1036EC0012434CEE75F009A42583F583E493900006
:1036FC0042F09008C675F009EF12434CEE75F009D4
:10370C00A42583F583E493900043F0900071A3E02B
:10371C009008C775F00912434CEE75F009A4258387
:10372C00F583E493FD900044F09008C875F009EF20
:10373C0012434CEE75F009A42583F583E4939000B5
:10374C0045F0900071A3E09008C975F00912434C44
:10375C00EE75F009A42583F583E493900046F09070
:10376C0008CA75F009EF12434CEE75F009A42583D5
:10377C00F583E493900047F0900071A3E09008CBA0
:10378C0075F00912434CEE75F009A42583F583E41A
:10379C0093900048F0ED6015900044E075F010A493
:1037AC0024B3F9740835F0FA7BFF12644590004598
:1037BC00E0FF601175F010A424B3F9740835F0FA29
:0E37CC007BFF126476900040E0900000F02237
:106041007BFF7A0D791A1264457BFF7A0D79FA127A
:1060510064767F0E121F32900005E0FF121F03903D
:106061000006E0FF121F037F1A121F3290003B74DB
:0F6071001AF090003C7404F09000007432F0229A
:10564E003028079000007403F0221264707F1E123F
:10565E001F321254C5900073E0FEA3E0FFD39400F6
:10566E00EE9400402FEF94FBEE9400502790003BF9
:10567E00741BF090003C7407F0900049743AF0E40B
:10568E0090004AF0900035E01490004BF09000002E
:0E569E007432F02212643F90000074FAF02281
:103BC400D3900072E09400900071E09400400A12D7
:103BD400643F90000074FAF022900071E0FEA3E0CC
:103BE400FF9008DC75F00912434CEE75F009A4252A
:103BF40083F583E493900040F09008DD75F009EFBD
:103C040012434CEE75F009A42583F583E4939000E8
:103C140041F0900071A3E09008DE75F00912434C66
:103C2400EE75F009A42583F583E493900042F090A7
:103C340008DF75F009EF12434CEE75F009A42583F3
:103C4400F583E493900043F0900071A3E09008E0C2
:103C540075F00912434CEE75F009A42583F583E44D
:103C640093FD900044F09008E175F009EF12434C85
:103C7400EE75F009A42583F583E493900045F09054
:103C84000071A3E09008E275F00912434CEE75F060
:103C940009A42583F583E493900046F09008E37526
:103CA400F009EF12434CEE75F009A42583F583E483
:103CB40093900047F0900071A3E09008E475F00938
:103CC40012434CEE75F009A42583F583E493900028
:103CD40048F0ED6015900044E075F010A424CCF990
:103CE400740835F0FA7BFF126445900045E0FF60EC
:103CF4001175F010A424CCF9740835F0FA7BFF1286
:0B3D04006476900040E0900000F02288
:105AAE0090003B741FF090003C7407F09000497416
:105ABE003AF0E490004AF0900038E090004BF07B12
:105ACE00FF7A0D792A1264451264707F0F121F320D
:105ADE00900005E0FF121F03900006E0FF121F0367
:0C5AEE007F1E121F329000007432F02264
:1037DA00125076D3900072E09400900071E0940049
:1037EA00400A12643F90000074FAF022900071E0DF
:1037FA00FEA3E0FF9008F575F00912434CEE75F050
:10380A0009A42583F583E493900040F09008F675A7
:10381A00F009EF12434CEE75F009A42583F583E411
:10382A0093900041F0900071A3E09008F775F009B9
:10383A0012434CEE75F009A42583F583E4939000B6
:10384A0042F09008F875F009EF12434CEE75F00952
:10385A00A42583F583E493900043F0900071A3E0DC
:10386A009008F975F00912434CEE75F009A4258306
:10387A00F583E493FD900044F09008FA75F009EF9F
:10388A0012434CEE75F009A42583F583E493900066
:10389A0045F0900071A3E09008FB75F00912434CC3
:1038AA00EE75F009A42583F583E493900046F09021
:1038BA0008FC75F009EF12434CEE75F009A4258354
:1038CA00F583E493900047F0900071A3E09008FD1F
:1038DA0075F00912434CEE75F009A42583F583E4CB
:1038EA0093900048F0ED6015900044E075F010A444
:1038FA0024E5F9740835F0FA7BFF12644590004517
:10390A00E0FF601175F010A424E5F9740835F0FAA7
:0E391A007BFF126476900040E0900000F022E7
:105AFA0090003B7424F090003C7407F090004974C5
:105B0A003AF0E490004AF0900039E090004BF07BC4
:105B1A00FF7A0D793A1264451264707F0F121F32B0
:105B2A00900005E0FF121F03900006E0FF121F031A
:0C5B3A007F1E121F329000007432F02217
:10392800125076D3900072E09400900071E09400F9
:10393800400A12643F90000074FAF022900071E08F
:10394800FEA3E0FF90095F75F00912434CEE75F095
:1039580009A42583F583E493900040F090096075ED
:10396800F009EF12434CEE75F009A42583F583E4C2
:1039780093900041F0900071A3E090096175F009FF
:1039880012434CEE75F009A42583F583E493900067
:1039980042F090096275F009EF12434CEE75F00998
:1039A800A42583F583E493900043F0900071A3E08D
:1039B80090096375F00912434CEE75F009A425834C
:1039C800F583E493FD900044F090096475F009EFE5
:1039D80012434CEE75F009A42583F583E493900017
:1039E80045F0900071A3E090096575F00912434C09
:1039F800EE75F009A42583F583E493900046F090D2
:103A0800096675F009EF12434CEE75F009A4258399
:103A1800F583E493900047F0900071A3E090096764
:103A280075F00912434CEE75F009A42583F583E47B
:103A380093900048F0ED6015900044E075F010A4F4
:103A4800244FF9740935F0FA7BFF1264459000455C
:103A5800E0FF601175F010A4244FF9740935F0FAED
:0E3A68007BFF126476900040E0900000F02298
:105B460090003B7429F090003C7407F09000497473
:105B56003AF0E490004AF090003AE090004BF07B77
:105B6600FF7A0D794A1264451264707F0D121F3256
:105B7600900005E0FF121F03900006E0FF121F03CE
:0C5B86007F1E121F329000007432F022CB
:103A7600125076D3900072E09400900071E09400AA
:103A8600400A12643F90000074FAF022900071E040
:103A9600FEA3E0FF9009C975F00912434CEE75F0DC
:103AA60009A42583F583E493900040F09009CA7534
:103AB600F009EF12434CEE75F009A42583F583E473
:103AC60093900041F0900071A3E09009CB75F00946
:103AD60012434CEE75F009A42583F583E493900018
:103AE60042F09009CC75F009EF12434CEE75F009DF
:103AF600A42583F583E493900043F0900071A3E03E
:103B06009009CD75F00912434CEE75F009A4258392
:103B1600F583E493FD900044F09009CE75F009EF2B
:103B260012434CEE75F009A42583F583E4939000C7
:103B360045F0900071A3E09009CF75F00912434C4F
:103B4600EE75F009A42583F583E493900046F09082
:103B560009D075F009EF12434CEE75F009A42583E0
:103B6600F583E493900047F0900071A3E09009D1AB
:103B760075F00912434CEE75F009A42583F583E42C
:103B860093900048F0ED6015900044E075F010A4A5
:103B960024B9F9740935F0FA7BFF126445900045A3
:103BA600E0FF601175F010A424B9F9740935F0FA34
:0E3BB6007BFF126476900040E0900000F02249
:106500003022079000007401F02290003B742EF0BE
:1065100090003C7407F07BFF7A0D795A12644512A3
:0E65200064707F1E121F329000007432F02251
:10622600302807900000742FF02290000AE06438AE
:106236006005A3E0B4390A12643F90000074FAF0D6
:10624600227BFF7A0E790A12644590000AE0540F09
:09625600F5489000007430F022BC
:105CBC0090000AE064386005A3E0B4390A12643F2E
:105CCC0090000074FAF0227BFF7A0D796A12644519
:105CDC0090000AE0540FF548D202D20A9000C8E0B6
:105CEC00F527122E177BFF7A0E793A126445C20201
:095CFC00C20A90000074FEF022BF
:105BDE0090000AE0540FF548302002D200122E2910
:105BEE0030201B201304E53B70F9122E20C2007BDF
:105BFE00FF7A0E793A12644590000074FEF030215F
:105C0E0019201104E53B70F9122E207BFF7A0E79D4
:0B5C1E003A12644590000074FEF02272
:10576500302356900001E0FF900034F0C223121F51
:1057750003900034E0FF1268635021900034E0FF8D
:1057850090003CE02403F582E43400F583EFF090CB
:10579500003CE004F0900000E004F022900034E0CA
:1057A500B42A079000007403F0227BFF7A0E791A61
:0A57B50012644590000074FAF0221F
:1052B00030236A900001E0FF900034F0C223121FF7
:1052C00003900034E0FFB42A0B90003BE090000014
:1052D000F0D22822EFB4230B90003BE0900000F0C6
:1052E000C22822900034E0FF1268635021900034FD
:1052F000E0FF90003CE02403F582E43400F583EF06
:10530000F090003CE004F0900000E004F0227BFF0D
:0E5310007A0E791A12644590000074FAF022A9
:105F7A0030233F900001E0FF900034F0121F03C26B
:105F8A0023900034E0FFB42A0B90003BE09000001D
:105F9A00F0D22822EFB4230B90003BE0900000F0EF
:105FAA00C228227BFF7A0E791A1264459000007487
:035FBA00FAF022D8
:0A596E00900043E0FF70033028387A
:10597800121F3212669F124A918F5E900041E052C8
:105988005EE55E60047F3180027F30121F0330289D
:1059980017C228E55E2430900023F090003374018C
:0859A800F090000074F0F02201
:0F59B000900046E0FF121F32900000E004F0224A
:105EF200302340900001E0FF900034F0C223121FD3
:105F020003900034E0FFB42A079000007403F022EB
:105F1200126863500F900034E090000DF090000082
:105F2200E004F0227BFF7A0E791A12644590000099
:045F320074FAF022EB
:10630700302332900001E0FF900034F0C223BF2A0F
:10631700079000007403F022900034E0B423079044
:106327000000E004F0227BFF7A0E791A1264459090
:06633700000074FAF022E0
:1057BF0012669F900075EEF0A3EFF0124A918F4F93
:1057CF0090003D7401F090000DE0B431089000415D
:1057DF00E0424F800E90000DE0B4301E900041E08B
:1057EF00F4524F900075E0FEA3E0FFAD4F124A5008
:1057FF001267C190000074FEF0227BFF7A0E791AB7
:0A580F0012644590000074FAF022C4
:10500100900043E0FF7003302856121F3212669F52
:10501100900075EEF0A3EFF0E4F54F900041E0FF52
:10502100E54FC39F5027900075E475F00112433698
:10503100AFF0FE124A918F507423254FF582E4346C
:1050410000F583E550F0121F03054F80CE30281084
:10505100C228E54F04900033F090000074F0F02274
:1050610090003C740AF0900046E0FF121F3290005D
:0550710000E004F02244
:104F8800302375900001E0FF900034F0C223121F17
:104F980003900034E0FFB42A079000007403F02265
:104FA800EFB42308900000E004F0803912686350E1
:104FB80038900034E0FF90003CE0FE04F074032ECB
:104FC800F582E43400F583EFF0900041E02409FF16
:104FD800E433FE90003CE0D39FEE6480F874809840
:104FE8004016900000E004F0227BFF7A0E791A1236
:094FF800644590000074FAF022F7
:10613B00302337900001E0FF900034F0C223121F90
:10614B0003900034E0FFB42A079000007403F022A0
:10615B00EFB42307900000E004F0227BFF7A0E7966
:0B616B001A12644590000074FAF02244
:1058700012669F900075EEF0A3EFF090003C740A62
:10588000F0E4F54F900041E0FFE54FC39F502790B3
:105890000075E475F001124336AFF0FE90003CE075
:1058A000FD04F074032DF582E43400F583E0FD126D
:1058B0004A50054F80CE7BFF7A0E793A12644590AC
:0658C000000074FEF0225E
:1052410030236B900001E0FF900034F0C223121F65
:1052510003900034E0FFB42A079000007403F022A9
:10526100126863501A900034E0FF90003CE0FE04A5
:10527100F074032EF582E43400F583EFF080107BA7
:10528100FF7A0E791A12644590000074FAF02290A8
:105291000041E02409FFE433FE90003CE0D39FEE9F
:0F52A1006480F87480984006900000E004F022CA
:1046F100900043E0FF700620280302479C121F32FE
:1047010012669F900075EEF0A3EFF0124A91122508
:10471100A7900041E0B4011090006EE0FF121F036A
:1047210090006EE0900023F0900041E0B4022090F0
:10473100006DE0FF121F0390006EE0FF121F039057
:10474100006DE0900023F090006EE0900024F09066
:104751000041E06403703090006CE0FF121F039091
:10476100006DE0FF121F0390006EE0FF121F039027
:10477100006CE0900023F090006DE0900024F09038
:10478100006EE0900025F0302811C228900041E031
:10479100900033F090000074F0F022900046E0FFAA
:1047A100121F3290003C740AF0900000E004F022E5
:105B92001225FD5002803B1225D58F4F900047E021
:105BA200FFE54FC39F402B900048E0FFE54FD39F96
:105BB200502012669F900075EEF0A3EFF0AD4F12E9
:105BC2004A507BFF7A0E793A12644590000074FEC7
:0C5BD200F02212643F90000074FAF022F0
:1059BF001225FD5002803F1225D58F4F900047E0F2
:1059CF00FFE54FC39F400B900048E0FFE54FD39F8B
:1059DF004004E54F702012669F900075EEF0A3EF24
:1059EF00F0AD4F124A507BFF7A0E793A1264459010
:1059FF00000074FEF02212643F90000074FAF0224F
:104D9500900043E0FF700330285E121F3212669FB9
:104DA500900075EEF0A3EFF0124A918F4F124C1060
:104DB500E4F54F746C254FF582E43400F583E0FF8C
:104DC5007423254FF582E43400F583EFF0746C25E8
:104DD5004FF582E43400F583E0FF121F03054FE52C
:104DE5004FC3940440CD30280FC22890003374037C
:104DF500F090000074F0F022900046E0FF121F32A0
:0D4E050090003C740AF0900000E004F022E0
:106080007F0A12437E8F4FE54F601212669F900089
:1060900075EEF0A3EFF0E54F14FD124A50E54F7B8B
:1060A000FF600E7A0E793A12644590000074FEF09B
:0F60B000227A0D79BA12644590000074FAF0223A
:10486300900043E0FF70062028030248FE121F3227
:1048730012669F900075EEF0A3EFF0124A91122595
:10488300A7900075E475F001124336AFF0FE124AAB
:104893009112258B90006DE0FF900023F0A3F0129E
:1048A3001F0390006EE0FF121F03900075E475F084
:1048B30001124336AFF0FE124A9112258B90006C21
:1048C300E0FF900025F090006DE0900026F090004E
:1048D3006EE0900027F0121F0390006DE0FF121F9F
:1048E3000390006EE0FF121F0330280FC2289000D0
:1048F300337405F090000074F0F022900046E0FF5E
:10490300121F3290003C740AF0900000E004F02281
:1047B10090000DE0540F75F00AA4FFA3E0540F2FF1
:1047C100F54F900010E0540F75F00AA4FF90000F10
:1047D100E0540F75F064A42FFF900011E0540F2FE7
:1047E100F550E54FC394014015E54FD39414500E95
:1047F100E550C394014007E550D394FA400A12648E
:104801003F90000074FAF02212669F900075EEF05E
:10481100A3EFF0900075E475F001124336AFF0FE9E
:10482100AD4F124A50900010E0540F75F00AA4FFEA
:1048310090000FE0540F75F064A42FFF900011E079
:10484100540F2FF54F900075E0FEA3E0FFAD4F121E
:104851004A507BFF7A0E793A12644590000074FE4B
:02486100F02243
:103D0F007F0D12437EEF701A900010E0B43010A3B5
:103D1F00E0B4300BA3E0B43006A3E06430600302DC
:103D2F003DF9900014E0FF64306004EFB4350E905D
:103D3F000015E0540FD394054003023DF990001491
:103D4F00E0FF64316004EFB43611900019E0B42045
:103D5F0007900018E0B42003023DF9900014E0FF33
:103D6F0064326004EFB43710900018E0B42007906D
:103D7F000017E0B420028072900014E0FF643360FB
:103D8F0004EFB43809900015E0B42002805C900075
:103D9F0014E0FF64346005EF64397058900015E04B
:103DAF00540F75F00AA4FFA3E0540F2FF54F9000A6
:103DBF0018E0540F75F00AA4FF900017E0540F7528
:103DCF00F064A42FFF900019E0540F2FF550E54F2A
:103DDF00C394014015E54FD39414500EE550C3948E
:103DEF00014007E550D394FA400A12643F90000057
:103DFF0074FAF02212669F900075EEF0A3EFF09028
:103E0F00003C740AF0E4F54F900041E0FFE54FC32A
:103E1F009F5027900075E475F001124336AFF0FE06
:103E2F0090003CE0FD04F074032DF582E43400F5BE
:103E3F0083E0FD124A50054F80CE7BFF7A0E793A10
:0A3E4F0012644590000074FEF0229A
:104F0C00900043E0FF700330285B121F3212669F43
:104F1C00900075EEF0A3EFF0E4F54F900041E0FF48
:104F2C00E54FC39F502C900075E475F00112433689
:104F3C00AFF0FE124A918F507423254FF582E43462
:104F4C0000F583E550F07E00124A91121F03054FC5
:104F5C0080C9302810C228E54F04900033F090002F
:104F6C000074F0F022900046E0FF121F3290003CDB
:0C4F7C00740AF0D226900000E004F0223D
:1053F400302365900001E0FF900034F0C223BF2AFF
:10540400079000007403F022900034E0FFB42308F6
:10541400900000E004F0803DEF547FFF121F0390E2
:105424000034E0547FFF90003CE0FE04F074032E4F
:10543400F582E43400F583EFF0900041E02409FFA5
:10544400E433FE90003CE0D39FEE6480F8748098CF
:095454004006900000E004F02283
:105A5F0030234B900001E0FF900034F0C223BF2AA7
:105A6F00079000007403F022900034E0FFB4230B82
:105A7F00900000E004F0E004F08010126863500F13
:105A8F00900034E090003EF0900000E004F0227BA4
:0F5A9F00FF7A0E791A12644590000074FAF02213
:1049B300202303024A4F900001E0FF900034F0C22D
:1049C30023BF2A079000007403F022900034E0FF15
:1049D300B4230A900000E004F0E004F022126863BC
:1049E300505B90003EE0540F75F00AA4FF90003432
:1049F300E0540F2FF0E0900C8693FF900034F012F8
:104A03001F03900034E0FF90003CE0FE04F07403C9
:104A13002EF582E43400F583EFF0900041E02409A1
:104A2300FFE433FE90003CE0D39FEE6480F8748093
:104A330098900000E0400304F02214F0227BFF7AF8
:0D4A43000E791A12644590000074FAF022FA
:106605003020099000DCE0F54D126720302203E4CC
:10661500F54D30210B301E05754D0A8003754D284B
:07662500900000E004F022E8
:10538A00E54D706512446C900040E012435853BAE0
:10539A006453BF6E53BF7853BF8253BF8C53C496B6
:1053AA0053C9A053CEAA53D3B453D8BE000053DB7B
:1053BA0012676B801C1264A18017126A168012127F
:1053CA006A17800D126A188008126A198003126A15
:1053DA001A30200F9000DEE09000A1F0900000E06B
:0A53EA0004F0229000007401F0228C
:106853009000A1E0700912673A9000007401F022E1
:1057090030200D9000DCE0F54D126720E54D70FC6E
:10571900302107754D05E54D70FCE4F54F30210C3E
:105729001268AF12255612692112255630200C1223
:1057390068BA122556126921122556054FE54FC33D
:10574900940540D930200E9000DEE09000A1F09041
:0C57590000A1E070FA9000007401F02242
:016A12002261
:016A13002260
:016A1400225F
:104E120030210A201E079000007401F02230200D7C
:104E22009000DCE0F54D126720E54D70FC30210763
:104E3200754D05E54D70FC30201B9000BFE0F52A52
:104E42001268BAE4F54F122556054FE54FC3940A8E
:104E520040F412692130211B9000C0E0F52A12684B
:104E6200AFE4F54F122556054FE54FC3940A40F4BF
:104E720012692130200E9000DEE09000A1F0900037
:0D4E8200A1E070FA121F6AE4900000F02217
:016A1500225E
:105FBD0030133E20233B9000A47464F0E542547FDF
:105FCD00FF900A7D93900001F030260EE54230E7F8
:105FDD0009EF900A8D93900001F0D223C213900027
:105FED0001E0B42307900002E004F022E4900002E7
:025FFD00F02290
:105FFF0030113E20233B9000A47464F0E540547FA1
:10600F00FF900A7D93900001F030260EE54030E7B7
:10601F0009EF900A8D93900001F0D223C2119000E6
:10602F0001E0B42307900002E004F022E4900002A4
:02603F00F0224D
:10291300202403022AC5302303022AC5900002E0C3
:10292300F552E4F09000A47464F0126A098F51D256
:1029330023E551B430079000017430F022E551B41F
:1029430031079000017431F022E551B43207900051
:10295300017432F022E551B433079000017433F06F
:1029630022E551B434079000017434F022E551B4E8
:1029730035079000017435F022E551B43607900015
:10298300017436F022E551B437079000017437F033
:1029930022E551B438079000017438F022E551B4B0
:1029A30039079000017439F022E551B423109000E7
:1029B300017423F0AF520552900002EFF022E5516B
:1029C300B42A07900001742AF022E551B44107901C
:1029D30000017441F022E551B442079000017442B2
:1029E300F022E551B443079000017443F022E5510E
:1029F300B464079000017444F022202603C223220A
:102A0300E551B461079000017461F022E551B462AD
:102A1300079000017462F022E551B463079000014E
:102A23007463F022E551B464079000017464F022EA
:102A3300E551B465079000017465F022E551B46671
:102A4300079000017466F022E551B4670790000116
:102A53007467F022E551B468079000017468F022AE
:102A6300E551B469079000017469F022E551B46A35
:102A730007900001746AF022E551B46B07900001DE
:102A8300746BF022E551B46C07900001746CF02272
:102A9300E551B46D07900001746DF022E551B46EF9
:102AA30007900001746EF022E551B46F07900001A6
:102AB300746FF022E551B470079000017470F02236
:032AC300C2232209
:0B687F007F209000037420F0A3DFFCDA
:01688A0022EB
:0F686300EFC394304007EFD39439500122C32282
:1050760090000CE0FD6420602E90000BE0540F754C
:10508600F00AA4FBAAF090000AE0540F75F064A49D
:105096002BFFE5F03AFEED540F7C002FFFEC3E901F
:1050A6000071F0A3EF803190000BE0FD64209000CA
:1050B6000A601AE0540F75F00AA4FFED540F7C0045
:1050C6002FFEEC35F0900071F0A3CE800BE0540F6C
:1050D600FF900071E4F0A3EFF0E024FFF090007180
:0550E600E034FFF022A0
:1054C500900009E0FD6420602B900008E0540F7502
:1054D500F00AA4FBAAF0900007E0540F75F064A44D
:1054E5002BFFE5F03AFEED540F7C002FFFEC3E90CC
:1054F5000073802E900008E0FD6420900007601A7C
:10550500E0540F75F00AA4FFED540F7C002FFEEC5C
:1055150035F0900073F0A3CEF022E0540FFF900019
:0755250073E4F0A3EFF02294
:1066C200900005E0540F75F00AA4FFA3E0540F2FC9
:1066D200900035F0D394004006E09415500122C397
:0166E2002295
:1056AC00E4FFEF75F003A4249DF582E4340AF5833E
:1056BC00E493FE900004E0FDEE6D703BEF75F0039B
:1056CC00A4249EF582E4340AF583E493FE9000054D
:1056DC00E0FDEEB50521EF75F003A4249FF582E4FF
:1056EC00340AF583E493FE900006E0FDEEB5050761
:0C56FC00900036EFF0D3220FBF33A7C39D
:01570800227E
:1055EE00E4FF75F003EFA42436F582E5F0340BF5F5
:1055FE0083E493FE900004E0FDEE6D703D75F003C4
:10560E00EFA42437F582E5F0340BF583E493FE9096
:10561E000005E0FDEEB5052275F003EFA42438F584
:10562E0082E5F0340BF583E493FE900006E0FDEE88
:0F563E00B50507900037EFF0D3220FBF70A4C35C
:01564D00223A
:10437E0074032FF582E43400F583E0FD6431706937
:10438E00FE74042FF582E43400F583E0FCEE75F044
:10439E0003A4249DF582E4340AF583E4936C704201
:1043AE0074052FF582E43400F583E0FCEE75F0031E
:1043BE00A4249EF582E4340AF583E493B5042374B1
:1043CE00062FF582E43400F583E0FCEE75F003A4CD
:1043DE00249FF582E4340AF583E493B50404EE04D5
:1043EE00FF220EBE339B7F0022ED6432706DFE7491
:1043FE00042FF582E43400F583E0FD75F003EEA49E
:10440E002436F582E5F0340BF583E4936D70457434
:10441E00052FF582E43400F583E0FD75F003EEA47C
:10442E002437F582E5F0340BF583E493B505257456
:10443E00062FF582E43400F583E0FD75F003EEA45B
:10444E002438F582E5F0340BF583E493B50505EEDB
:0D445E002434FF220EBE70977F00227F00E5
:01446B00222E
:104C1000EFC3943390006C50397431F0EF75F003AA
:104C2000A4249DF582E4340AF583E49390006DF0AA
:104C3000EF75F003A4249EF582E4340AF583E4932F
:104C400090006EF0EF75F003A4249FF582E4340A1F
:104C5000803A7432F075F003EFA4249DF582E5F0FC
:104C6000340AF583E49390006DF075F003EFA4240B
:104C70009EF582E5F0340AF583E49390006EF075BA
:104C8000F003EFA4249FF582E5F0340AF583E49362
:054C900090006FF0220E
:10678200900005E0540F75F00AA4FFA3E0540F2F08
:05679200900038F02228
:10679700900005E0540F75F00AA4FFA3E0540F2FF3
:0567A700900039F02212
:1067AC00900005E0540F75F00AA4FFA3E0540F2FDE
:0567BC0090003AF022FC
:10669F0090004BE0FF90004AE08FF0A4FF9000497C
:1066AF00E07C002FFFEC35F0FE900042E02FFFEC76
:0366BF003EFE227A
:1067C100900044E075F010A4244DF9740235F0FAFC
:0567D1007BFF0264766D
:036A09007F0322E6
:10676B00302008900023E0FF12689730210890003A
:07677B0023E0FF12688B22EE
:1064A100E4F55E900033E0FFE55EC39F5021742365
:1064B100255EF582E43400F583E0F55F302004FFCA
:0F64C100126897302105AF5F12688B055E80D49B
:0164D00022A9
:016A1600225D
:016A1700225C
:016A1800225B
:016A1900225A
:016A1A002259
:0C688B001268C512255612692802255615
:0C6897001268D0122556126928022556FE
:10446C00E4F55EF55FF560900072E02401FF9000CA
:10447C0071E03400FEC3EF940AEE94005005A3E003
:10448C0004F560D3EF9463EE9400404C900072E01E
:10449C002401FB900071E03400FA7C007D64AF03D2
:1044AC00FE1242E18F5EEF75F064A4FFC3EB9FFF39
:1044BC00EA95F0FE7C007D0A1242E18F5FA3E004D6
:1044CC00FFE55E75F064A4FEC3EF9EFFE55F75F03B
:1044DC000AA4FEC3EF9EF560900072E02401FF90E9
:1044EC000071E03400FED3EF9409EE940040197C87
:1044FC00007D0A1242E18F5FA3E004FFE55F75F0D7
:10450C000AA4FEC3EF9EF5607430255EF55E743030
:10451C00255FF55F74302560F560302014AF5E12B6
:10452C006897AF5F126897AF601268977F2A12681E
:10453C0097302114AF5E12688BAF5F12688BAF603F
:08454C0012688B7F2A12688BB4
:014554002244
:06643F007BFF7A0D798A53
:066445008B5F8A60896193
:10644B007F01121F32E4F562AB5FAA60A96185621E
:10645B00827583001242A2FF121F030562E562C31D
:04646B00941040E465
:01646F00220A
:066470007BFF7A0D79DAD2
:066476008B608A6189625F
:10647C007F11121F32E4F563AB60AA61A9628563D8
:10648C00827583001242A2FF121F030563E563C3EA
:04649C00941040E434
:0164A00022D9
:1060BF007BFF7A0E794A1264761261ECE4F55EF595
:1060CF005FE55F900A3C93FDAF5FAE5E124A50E50D
:1060DF005F900A3C93FDAF5FAE5E125D05055FE515
:0E60EF005F7002055EC3943AE55E940040D3F4
:0160FD002280
:016A1B002258
:016A1C002257
:016A1D002256
:016A1E002255
:016A1F002254
:016A20002253
:016A21002252
:10662C007BFF7A0E79CA1264451260BF126A1B1284
:10663C006A1C126A1D126A1E126A1F126A20126AE2
:07664C0021121F4C021F5B2D
:1064D100755E01755F007560B3E4F561AF617E00C3
:1064E100124A91AB5E0560E560AA5F7002055F1418
:0E64F100F9EF1242CF0561E561C3943A40DE37
:0164FF00227A
:1065B4001261ECE4F55EF55FAF5FAE5E124A91AD39
:1065C40007AF5FAE5E125D05055FE55F7002055EB5
:0965D400C3943AE55E940040DF37
:0165DD00229B
:10665300E4F564F565AF65AE6412652EAD07AF650D
:10666300AE64124A500565E56570020564C3943A49
:06667300E564940040DF25
:0166790022FE
:10625F00755E01755F007560B3E4F561F562AF625D
:10626F00AE6112652EAB5E0560E560AA5F70020538
:10627F005F14F9EF1242CF0562E56270020561C348
:08628F00943AE561940040D649
:0162970022E4
:10629800755E01755F007560B3E4F561F562AB5E2C
:1062A8000560E560AA5F7002055F14F9124289FD76
:1062B800AF62AE61124A500562E56270020561C3C1
:0862C800943AE561940040D610
:0162D00022AB
:104A5000C2B0758400D2C2C2C6D2C6C2C4D2C5C258
:104A6000C330C3FD74A0F5C2C2C5C2C330C3FD8E3E
:104A7000C2C2C330C3FD8FC2C2C330C3FD8DC2C228
:104A8000C330C3FDD2C4C2C320C4FD12253ED2B080
:104A900022758400C2C3D2C530C3FD74A0F5C2C262
:104AA000C5C2C330C3FD8EC2C2C330C3FD8FC2C2F4
:104AB000C330C3FDC2C4D2C5C2C330C3FD74A1F5A7
:104AC000C2C2C5C2C330C3FDC2C2C2C330C3FD85AA
:104AD000C207D2C4C2C320C4FD22D2C2C2C6D2C63B
:084AE000D2C4C2C320C4FD22B0
:102E1700754700122E3250FB22754700122EBB5009
:102E2700FB22754700122E7250FB22758400E5477E
:102E370075F003A4902E3F73022ED7022EE6022FC1
:102E470004022EED022F10022F17022F1F022EE66B
:102E5700022F2D022EED022F3D022F46022ED70202
:102E67002EE6022F54022EED022F60758400E547EF
:102E770075F003A4902E7F73022ED7022EE6022F41
:102E870004022EED022F10022F17022ED7022EE674
:102E9700022F04022EED022F10022F17022F10020D
:102EA7002F17022F1F022EE6022F62022EED022F8E
:102EB7003D022F60758400E54775F003A4902EC886
:102EC70073022ED7022EE6022F54022EED022F6038
:102ED700C2FA122F72122F72759B000547C3223058
:102EE700F9020547C32230F912E59A20E7FB122FB2
:102EF70072D2FA122F72122F720547C322C2FA1228
:102F07002F72759B040547C322753A1E0547C322D6
:102F1700E53A70020547C322C2FA122F72122F93A5
:102F2700F59B0547C322C2FA122F72122FA244073C
:102F3700F59B0547C322122F84F53B0547C322752E
:102F4700840F30DE04E53B70020547C322C2FA1244
:102F57002F72759B080547C322D322C2FA122F721C
:092F6700122FA24405F59B054759
:102F7000C32200000000000000000000000000006C
:102F800000000022902F8BE54893225A5A5A5A5A31
:102F9000FAFAFA902F9AE548932200B45AE12D8765
:102FA0007ADB902FA9E54893220000000000008002
:012FB00080A0
:105F36002A2A3132333435362A2A2A2A3132333460
:105F460035302A2A44313233343536373839302A17
:105F560023414243202056455253494F4E20322E6C
:105F660031332000202020205349454D454E5320F3
:045F760020202020A7
:104C9500302920C229E542540F905F4A9390008C39
:104CA500F0786876329000B4E06015126372126194
:104CB500B1800D7868E67008900078F0900089F072
:104CC500302A3EC22AE540540F905F4A9390008BEC
:104CD500F0754A32125D4E301E06740044B37009F9
:104CE500201E099000B5E06003126176301E06743F
:104CF5000044B37003201E0312633D201E1302639C
:104D0500DBE54A700C900079F0900088F09000ED9A
:024D1500F0228A
:10633D00900079E0FF04F0EF905F3693FF90008BB3
:10634D00E0FEEF6E6011EEB42A089000797401F052
:10635D008005E4900079F0900079E0B40A06E4F04D
:05636D00D221D22B2219
:10637200900078E0FF04F0EF905F3693FF90008C7E
:10638200E0FEEF6E6011EEB42A089000787401F01E
:106392008005E4900078F0900078E0B40A06E4F01A
:0563A200D220D22B22E5
:10617600900088E0FF04F0747F2FF582E43400F588
:1061860083E0FF90008BE0FEEF6E6011EEB4230813
:106196009000887401F08005E4900088F0900088F3
:0B61A600E0B40906E4F0D221D21F2271
:1061B100900089E0FF04F0747F2FF582E43400F54C
:1061C10083E0FF90008CE0FEEF6E6011EEB42308D7
:1061D1009000897401F08005E4900089F0900089B5
:0B61E100E0B40906E4F0D220D21F2237
:1063DB0090007BE0FF04F0EF905F4093FF90008B09
:1063EB00E0FEEF6E6011EEB42A0890007B7401F0B2
:1063FB008005E490007BF090007BE0B40A04E4F0AD
:03640B00D22C226E
:10655C0090007F7423F0A3F0E4FF74B72FF582E46E
:10656C003400F583E0FE74812FF582E43400F5836A
:0C657C00EEF00FBF06E49000877423F0DF
:0165880022F0
:105A0F00121E60121F4C7F01121F327BFF7A5F79CB
:105A1F006A1264457BFF7A5F795A1264767539147E
:105A2F00E490007EF090007DF0FF744C2FF582E43F
:105A3F003400F583E4F0745C2FF582E43400F583D1
:105A4F00E4F00FBF10E4E53970FC121F4C021F5B2E
:1051D00090007EE0FFD3940F501FEF04FF121F32A8
:1051E00090008BE0FF90007EE0FE04F0744C2EF502
:1051F00082E43400F583EF80437F01121F32E4F52F
:105200005E744D255EF582E43400F583E0FF744C56
:10521000255EF582E43400F583EFF0744C255EF5ED
:1052200082E43400F583E0FF121F03055EE55EC3F0
:10523000940F40CD90008BE0FF90005BF0121F03B5
:01524000224B
:10515E0090007DE0FFD3940F5020EF2411FF121F1B
:10516E003290008CE0FF90007DE0FE04F0745C2E27
:10517E00F582E43400F583EF80437F11121F32E491
:10518E00F55E745D255EF582E43400F583E0FF7410
:10519E005C255EF582E43400F583EFF0745C255EE9
:1051AE00F582E43400F583E0FF121F03055EE55E31
:1051BE00C3940F40CD90008CE0FF90006BF0121F57
:0151CE0003DD
:0151CF0022BD
:105D4E009000EDE0FF700E90008BE0B42A079000FB
:105D5E00ED7401F022EFB4011390008BE0B4230731
:105D6E009000ED7402F022E49000EDF09000EDE072
:105D7E00B4021490008BE0B430089000EE7401F081
:085D8E008000E49000EDF0221A
:10455500E53760021537E53A6002153A900093E0B9
:10456500600214F0900097E0600214F090009BE068
:10457500600214F090009FE0600214F09000A2E049
:10458500600214F09000AAE0600214F09000B2E01E
:10459500600214F022E538600215389000A1E06051
:1045A5000214F0900092E0600214F0900096E06032
:1045B5000214F09000A7E0600214F022E5396002D1
:1045C5001539E53B6002153BE54C6002154CE54DA0
:1045D5006002154D7868E6600116E54A6002154AE5
:1045E500E54B6002154B9000AFE0600214F09000BF
:1045F5009AE0600214F090009EE0600214F09000D2
:10460500A8E0600214F09000EFE0600214F02222AE
:104615009000A4E0600214F0229000A3E060021470
:02462500F02281
:1020AA00202046554E4354494F4E20313820202097
:1020BA0000202020454D455247454E4359202020B7
:1020CA002000202020205354414E444259202020F1
:1020DA002020524144494F204F524947494E4154CA
:1020EA00452054454C434F204F524947494E41548D
:1020FA00452020202046554E4354494F4E2031203A
:10210A00202020202046554E4354494F4E2032204D
:10211A00202020202046554E4354494F4E2033203C
:10212A00202020202046554E4354494F4E2034202B
:10213A00202020202046554E4354494F4E2035201A
:10214A00202020202046554E4354494F4E20362009
:10215A00202020202046554E4354494F4E203720F8
:10216A00202020202046554E4354494F4E203820E7
:10217A00202020202046554E4354494F4E203920D6
:10218A002020202052454345495645204D4F44457D
:10219A002020205452414E534D4954204D4F44451E
:1021AA002020202046554E4354494F4E203130209E
:1021BA002020202046554E4354494F4E203131208D
:1021CA002020202046554E4354494F4E203132207C
:1021DA002020202046554E4354494F4E203133206B
:1021EA002020202046554E4354494F4E203134205A
:1021FA002020202046554E4354494F4E2031352049
:10220A002020202046554E4354494F4E2031362037
:10221A002020202046554E4354494F4E2031372026
:10222A002020202046554E4354494F4E2031382015
:10223A002020202046554E4354494F4E2031392004
:10224A002020202046554E4354494F4E20323020FC
:10225A002020202046554E4354494F4E20323120EB
:10226A002020202046554E4354494F4E20323220DA
:10227A002020202046554E4354494F4E20323320C9
:10228A002020202046554E4354494F4E20323420B8
:10229A002020202046554E4354494F4E20323520A7
:1022AA002020202046554E4354494F4E2032362096
:1022BA002020202046554E4354494F4E2032372085
:1022CA0020203A0036AA340031552EAA2C0029556E
:0E22DA0026AB240021551EAB1C001955140024
:101B75009000E8E07003021E5F202D0F9000B0E09A
:101B850060099000AFE07003021E5B202D03021E6A
:101B95005FC22D9000B0E0FF701DE540B40B0C90C6
:101BA50000AF7414F09000B0E004F0E540640C6000
:101BB50003021E5F021DD5EF64016003021CC8E528
:101BC50040B40B03021D7BE540B40C0D9000AF74CF
:101BD50014F09000B07404F0229000DBE0C394038D
:101BE500502EE54094004028E54094085022E540F9
:101BF500149000ACF09000AE7401F09000ACE0756C
:101C0500F010A424FCF9742035F0FA7BFF1264452A
:101C15009000DBE0B4032FE540D394074028E5406E
:101C2500940A5022E540149000ACF09000AE740187
:101C3500F09000ACE075F010A424FCF9742035F0A8
:101C4500FA7BFF1264459000DBE064047035E540E3
:101C55006408702F7BFF7A21796C1264457BFF7ACB
:101C650021799C1264769000EBE0B4030312692F8E
:101C75009000ECE0B4030312693B1267209000B1B9
:101C85007401F09000DBE064047034E54064097091
:101C95002E7BFF7A21797C1264457BFF7A21798C32
:101CA5001264769000EBE0B403031269359000EC02
:101CB500E0B4030312694112673AE49000B1F0E41D
:101CC500021E5B9000B0E064036003021D6EE540F8
:101CD500B40C129000AF7414F0E49000F4F090008E
:101CE500B07405F022E540B40B03021DE7E540B4EE
:101CF500092E9000ACE09000ADF09000AC7414F0AB
:101D0500E49000ABF09000AE04F07BFF7A2079AA56
:101D15001264457BFF7A2079BB126476E4021E5B70
:101D25009000DBE0C394035007E540C394084005E9
:101D3500E540B40A30E540B40A089000AC7409F0F7
:101D45008008E54024099000ACF09000AE7401F0E5
:101D55009000ACE075F010A4241CF9742135F0FA5C
:101D65007BFF126445E4021E5B9000B0E0640470E2
:101D75004FE540B40C079000AF7414F022E540B471
:101D85000B02805E9000DBE0C39403502FE5409486
:101D9500004029E540940A5023E54024149000AC06
:101DA500F09000AE7401F09000ACE075F010A42442
:101DB500ECF9742035F0FA7BFF126445E4021E5BF2
:101DC5009000B0E064056003021E5FE540B40C0DB1
:101DD5009000AF7414F09000B07403F022E540B4A5
:101DE5000B0D9000AF7414F09000B07401F02290C8
:101DF50000DBE0C39403505DE540C3940B5056905F
:101E050000AF7414F0E5409000F4B40A12E0FF044A
:101E1500F074F02FF582E43400F583E4F08011E0EE
:101E2500FF04F074F02FF582E43400F583E540F00B
:101E35009000F4E0D3940340219000F0E094085022
:101E45000E9000F2E0C3940850051267D680031285
:0B1E55006702E48001E49000B0F0227E
:1017D5009000DBE064047003021B749000AEE070BF
:1017E50003021B741269D39000ABE0FF70309000C8
:1017F500ACE0FE64076011EEC39405400BEED39494
:1018050013400CEE941850079000AB7401F022EED3
:101815009000ABB408047408F0227404F022EFB40D
:1018250001030219599000ABE0640260030218E05D
:101835009000AAE06003021B749000ACE0FF600317
:10184500B4070C9022D0E493F516740193F517EFC5
:10185500B4010C9022D2E493F516740193F517EFB9
:10186500B4020C9022DCE493F516740193F517EF9E
:10187500B4030C9022DEE493F516740193F517EF8B
:10188500B4040C9022D8E493F516740193F517EF80
:10189500B4140C9022CEE493F516740193F517EF6A
:1018A500B4150C9022DAE493F516740193F517EF4D
:1018B500B4160C9022D4E493F516740193F517EF42
:1018C500B4170C9022D6E493F516740193F517908E
:1018D50000C4E0F5281269D9021A569000ABE064FD
:1018E50003706A9000AAE06003021B749022CC93F7
:1018F500F516740193F5179000C5E0F5281269D91E
:101905009000B17401F01269B5E49000ABF090005D
:10191500AEF09000ACE064146003021B749000AD5F
:10192500E09000ACF01269DC121F4CE49000B1F0BD
:1019350090009CF0900099F09000DEE0FF9000D9B7
:10194500E02F9000A1F09000A5740AF0229000AB62
:10195500E0B404209022CCE493F516740193F517B6
:101965009000C6E0F5281269D91269D39000AA74CF
:1019750078021B269000ABE0FF64056003021A5E47
:101985009000AAE06003021B749000ACE0FEB40571
:101995000C9022E0E493F516740193F517EEB40666
:1019A5000C9022E2E493F516740193F517EE6409A1
:1019B5006004EEB4180C9022E0E493F516740193DC
:1019C500F517EE640A6004EEB4190C9022E0E49376
:1019D500F516740193F517EE640B6004EEB41A0C5A
:1019E5009022E0E493F516740193F517EEB40C0C10
:1019F5009022E0E493F516740193F517EEB40D0CFF
:101A05009022E2E493F516740193F517EE640E60E7
:101A150004EEB41B0C9022E2E493F516740193F5E1
:101A250017EE640F6004EEB41C0C9022E2E493F50B
:101A350016740193F517EE64106004EEB41D0C9056
:101A450022E2E493F516740193F5179000C4E0F5CE
:101A5500289000AA7428021B26EF64066003021B67
:101A65002E9000AAE06003021B749000ACE0FF64B6
:101A7500056004EFB4060C9022D0E493F5167401CA
:101A850093F517EF64096004EFB40D0C9022D2E4CE
:101A950093F516740193F517EF640A6004EFB40E1D
:101AA5000C9022DCE493F516740193F517EF640BA3
:101AB5006004EFB40F0C9022DEE493F516740193E5
:101AC500F517EF640C6004EFB4100C9022D8E49382
:101AD500F516740193F517EF64186004EFB41B0C49
:101AE5009022DAE493F516740193F517EF64196003
:101AF50004EFB41C0C9022D4E493F516740193F50D
:101B050017EF641A6004EFB41D0C9022D6E493F528
:101B150016740193F5179000C4E0F5289000AA7497
:101B250028F09000ABE004F0229000ABE0FFB40792
:101B3500279000AAE070389022CC93F51674019393
:101B4500F5179000C5E0F5289000B17401F0E49018
:101B550000ABF09000AEF022EFB408131269DC126E
:101B650069D6E49000ABF09000AEF09000B1F022A1
:10251200000000000000000000000000000022C0D7
:1025220000C001790478B4D8FED9FAD001D00022D3
:10253200C0007814122521D8FBD00022C0E07537E4
:1025420005E53770FCD0E022C0E075370FE5377043
:10255200FCD0E022C0E0753764E53770FCD0E022A1
:10256200A42582F582E58335F0F58322B40A0022A0
:10257200C0E0C3997001D3D0E022B5060122500712
:10258200B5070122400122D322EF75F06484243082
:1025920090006CF0E5F0A375F00A842430F0A3E516
:1025A200F02430F022EF75F06484243090006CF057
:1025B200E5F0A375F00A842430F0A3E5F02430F0AE
:1025C20090006CE0B4300B7420F0A3E0B4300374DC
:1025D20020F02290000DE0540FFFA3E0B42002800F
:1025E20019540FCF75F00AA42FFFA3E0B420028084
:1025F20009540FCF75F00AA42FFF22C006C005C0F0
:082602000490000DE0540FFFED
:10260A00FEA3E0B42003C3802C540FFDCF75F00A5B
:10261A00A42FFFA3E0B42003C3801A540FFCEE7565
:10262A00F064A420D20EFEED75F00AA42E40052C0B
:10263A0040028001D3D004D005D0062275F064840C
:10264A00F6E5F00875F00A84F608A6F00822C0013B
:10265A007900E6B4FF028027F908E6B4FF03C380D5
:10266A0022E975F00AA426F908E6B4FF03C3801329
:10267A00E975F00AA420D207C3264003F98004D3DF
:10268A00D00122E9D00122E675F00AA408262278B0
:10269A0047EE12264675450075460078499026F29F
:1026AA007908EF134007A3A3A3A3A3801CC0E0C02B
:1026BA0000C001C37905E49336D4A2E4540FF6A30B
:1026CA0018D9F3D001D000D0E0D9D8E545600C750F
:1026DA004609754709754809754909854645854773
:1026EA004685484785494822060502000002010539
:1026FA0000000402000100080400020006090004A8
:10270A00000209010800040803060108060702037B
:1022E80020205455524E204F4E2053572020202056
:1022F8000020205455524E204F4646205357202048
:10230800200044313233343536373839302A2341C6
:10231800424302AB055508000AAB0D55100012AB3D
:10232800155518001AAB1D55200022AB255528005D
:102338002AAB2D55300032AA355520205445535428
:1023480020524F5554494E4520202020564552537F
:10235800494F4E20312E30202020205445535449D7
:102368004E4720454550524F4D2020205445535448
:10237800494E4720564F4943452020544553544918
:102388004E472044544D462031202054455354494B
:102398004E472044544D4620322020205445535463
:1023A800494E47205253323332202020544553544B
:1023B800494E472052533438352020202054455365
:1023C80054494E47205054542020205445535420FB
:1023D8004155582052454C415920205445535420CA
:1023E80043542052454C4159202020544553494ECE
:1023F800472052494E47494E472020202020202080
:102408002020202020202020202020544553542004
:102418004C494E452052414C415954455354204C47
:10242800494E452053454E53452B54455354204C53
:10243800494E452053454E53452D2020544553546D
:10244800204449475F494E202020205445535420BA
:10245800494E50555420564F4C54205445535420FF
:102468004C494E452052454C415954455354205AE5
:1024780045524F2043524F53532054455354494ECD
:102488004720535155454C43482020205445535428
:10249800494E472048504620202020544553542078
:1024A80054454C434F20564F5820205445535420F0
:1024B800524144494F20564F5820205445535420E8
:1024C800454D5F4F505450202020202020202020B0
:1024D80020202020202020202020202020202020F4
:1024E8002020202020202020202020544553542024
:1024F800434F4D504C4554454420202020544553CB
:0A25080054204641494C4544202070
:100EDA007BFF7A2379421264457BFF7A2379521287
:100EEA0064761268F17BFF7A237962126445121FD5
:100EFA005B1268F17F007E00124A918F4F7DAA7FB4
:100F0A00007E00124A507F007E00124A91EF64AAC6
:100F1A00600C7BFF7A257902126476126A0C7D5581
:100F2A007F007E00124A507F007E00124A91EF64D1
:100F3A0055600C7BFF7A257902126476126A0CAD31
:100F4A004F7F007E00124A507BFF7A2479F21264A6
:100F5A00451268F17BFF7A23797212644512694D52
:100F6A001268AF754700754801753914122E29E5C4
:100F7A003970FC122E20126989754700754801756F
:100F8A003905E53970FCD202D20A122E17C202C202
:100F9A000A7BFF7A2479F21264451268F17BFF7AA0
:100FAA00237982126445121F5B1268F17F3112683D
:100FBA00D0753932E53970FC1269283013FD12698F
:100FCA0028E542547FFFEF90230A93FFEFB4310ED6
:100FDA007BFF7A2479F21264451268F1800C7BFF58
:100FEA007A257902126476126A0C7BFF7A23799247
:100FFA00126445121F5B1268F17F311268C51268CC
:10100A00F91269283011FDE540547FFFEF90230A59
:10101A0093FFEFB4310E7BFF7A2479F21264451202
:10102A0068F1800C7BFF7A257902126476126A0CC9
:10103A007BFF7A2379A2126445121F5B1268F1754D
:10104A008400759850C299C2987599433098FD7575
:10105A008400E5996443600C7BFF7A257902126467
:10106A0076126A0C7BFF7A2479F21264451268F1CF
:10107A007BFF7A2379B2126445121F5B1268F11260
:10108A006991758400759850C299C29875994330D0
:10109A0099FD7BFF7A2479F21264451268F17BFF8D
:1010AA007A2379C2126445121F5B1268F112672013
:1010BA001268F9E53ED39432400C7BFF7A25790217
:1010CA00126476126A0C12673A1268F9E53EC39402
:1010DA00AA500C7BFF7A257902126476126A0C7B7D
:1010EA00FF7A2479F21264451268F17BFF7A237938
:1010FA00D2126445121F5B1268F112692F1268F945
:10110A00E53DD3940A400C7BFF7A25790212647676
:10111A00126A0C1269351268F9E53DC394AA500C9B
:10112A007BFF7A257902126476126A0C7BFF7A2495
:10113A0079F21264451268F17BFF7A2379E212642C
:10114A0045121F5B1268F112693B1268F11268F1CD
:10115A001269417BFF7A2479F21264451268F17BA5
:10116A00FF7A247912126445121F5B1268F1126920
:10117A00471268F11268F112694D1268F11268F1AA
:10118A007BFF7A247942126445121F5B1268F130A0
:10119A00DC1D7BFF7A2279E812647620DCFD121FBF
:1011AA005B7BFF7A2479F21264451268F1801B7B1B
:1011BA00FF7A2279F912647630DCFD121F5B7BFF1D
:1011CA007A2479F21264451268F17BFF7A2479C293
:1011DA00126445121F5B1268F1126971501F7BFF7E
:1011EA007A2279E812647612697140FB121F5B7BDE
:1011FA00FF7A2479F21264451268F1801D7BFF7A26
:10120A002279F912647612697150FB121F5B7BFF17
:10121A007A2479F21264451268F17BFF7A247952B2
:10122A00126445121F5B1268F1E53CC3940A400739
:10123A00E53CD39446400C7BFF7A2579021264760A
:10124A00126A0C7BFF7A2479F21264451268F17BE8
:10125A00FF7A247972126445121F5B1268F11268D0
:10126A00DB1269AC40FB1269AC50FB1269AC40FB63
:10127A007BFF7A2479F21264451268F11269217BA4
:10128A00FF7A247982126445121F5B1268F112698F
:10129A0053400F12672012673A12695350F58002C1
:1012AA0080F17BFF7A2479F21264451268F17BFFA0
:1012BA007A2479B2126445121F5B1268F11268E649
:1012CA0012695950FB800280F71269217BFF7A2448
:1012DA0079F21264451268F17BFF7A2479921264DA
:1012EA0045121F5B1268F11268DB12690190231C18
:1012FA00E493F508740193F50912690190231EE439
:10130A0093F508740193F509126901902320E49377
:10131A00F508740193F509126901902322E493F503
:10132A0008740193F509126901902324E493F508DE
:10133A00740193F509126901902326E493F5087460
:10134A000193F509126901902328E493F5087401C1
:10135A0093F50912690190232AE493F5087401931D
:10136A00F50912690190232CE493F508740193F5A9
:10137A000912690190232EE493F508740193F50983
:10138A00126901902330E493F508740193F5091268
:10139A006901902332E493F508740193F5091269FF
:1013AA0001902334E493F508740193F50912690155
:1013BA00902336E493F508740193F50912690190B4
:1013CA002338E493F508740193F50912690190230F
:1013DA003AE493F508740193F50912690190233CE4
:1013EA00E493F508740193F50912690190233EE428
:1013FA0093F508740193F509126901902340E49367
:10140A00F508740193F5091269217BFF7A2479F2B0
:09141A001264451268F10212F19E
:0114230022A6
:0868F10075390AE53970FC223B
:0868F900753902E53970FC223B
:08690100753905E53970FC222F
:036A0C0080FE22E7
:08000300022AC6000000000003
:08000B00022AC70000000000FA
:08001300022BFA0000000000BE
:08001B003200000000000000AB
:09002300320000000000000000A2
:08002B00022ACA0000000000D7
:08003300320000000000000093
:0A003B003200000000000000000089
:0900430032000000000000000082
:08004B0032000000000000007B
:08005300320000000000000073
:08005B00022B2C000000000044
:08006300320000000000000063
:08006B00022B4B000000000015
:08007300022AD0000000000089
:08007B00022BFB000000000055
:08008300022B2900000000001F
:08008B0032000000000000003B
:10009300022C190000000000000000000000000016
:1000A3003275FF0775FFDE75FFAD75840F75E107C8
:1000B30075E20475E34475840F75A43575A5097558
:1000C300A6FF75A7FF759CFF759D00759E00759F24
:1000D300F075D8FF75E8FF75F80F75AD0F758401DE
:1000E30075893075888F75840275893075888F7529
:1000F300840F758A80758C67780874FF0000000090
:100103000000000000000000D5E0F1D8EDE58C30E0
:10011300E7FB759701758A0043890475840075B7F9
:100123001075840F438901758D01758F01758E02DA
:100133007480D5E0FD438902E58930E4FB759702BD
:1001430075840075D10775840075BB0175BA007598
:10015300BCF075C70075C60075C5FF75C4FF75E8AB
:100163008175840275BB0475BA0075BCF175C60050
:1001730075C4FF75E88875840075D484758401752A
:10018300D484758400C2F8759A47759D1A43F8099B
:1001930075870075840075B90075A90075910075A0
:1001A300985075840175981075840075C04075C3A7
:1001B3000075CFC9758400758E0075892075880513
:1001C300758400758A00758B6F758CF4758D6F431C
:1001D300885075840075C90075CA0075CB0075CC4D
:1001E3000075CD0075840175C91875CA8075CBFB80
:1001F30075CDFB75CC80D2CA75840275C91875CAD2
:10020300A675CBAF75CDAF75CCA6D2CA7584007574
:10021300A8AF75B80075E6A475E71775F60075F70E
:10022300019000007F007E20E4F0A3DFFCDEFA757E
:0202330027FFA3
:100235007528FF7529FF752AFF752BFF752CFF752E
:080245002DFFD2B6124ADA22A5
:105D0500AC84A2AF922EABB1C2AF75840F53A1FE86
:105D150075B121E4F58443B701F584438F01786CAF
:105D2500768008F6EF26F618EE36F6E6FE08E6F576
:105D3500828E83EDF0E4F584538FFEF58453B7FE30
:085D45008BB18C84A22E92AFF9
:015D4D002233
:10652E00AD84A2AF922EACB1C2AF75B121756680AB
:10653E00756700EF2567F567EE3566F56685678248
:0D654E00F583E493FF8CB18D84A22E92AFF3
:01655B00221D
:1061EC00AF84A2AF922EAEB1C2AF786C7680087637
:1061FC000075B121E4F58443B701F584758F03185C
:10620C00E6FC08E6F5828C83E4F0F58FF58453B751
:09621C00FE8EB18F84A22E92AF18
:016225002256
:1049130008D0094E09D40A600AF40B910C360CE551
:104923000D9D0E600F2D100610EB11DD12DC13EA46
:1049330015071633177118C01D2107B107E80820A2
:104943000859196E1A211ADA1B971C5A0894090E72
:1049530009900A190AA90B410BE30C8C0D3F0DFDBD
:104963000EC50F9810771162125B13621477159BB3
:1049730016D018161DEF1EC21F9B2079215F224AF5
:10498300233B2434253326392747285C29792A9D5C
:104993002BC92CFE2E3B2F8230D032293379350A96
:1049A300367F3641397B3AFE3C943E41400741D144
:0F68210075F00212434CE493F508740193F509E6
:03683000D215225C
:036A0F00C215228B
:0869090075391EE53970FC220E
:08691100753950E53970FC22D4
:08691900753864E53870FC22BA
:104E8F00126A0F9000F0E0540F75F014A42413F57C
:104E9F0082E43449F583C083C0829000F1E0540F5F
:104EAF00D082D0831268219000F2E0540FFF90005F
:104EBF00F0E0540FB507159000F3E0540FFF90008A
:104ECF00F1E0540FB50705126911802D12691912FF
:104EDF006A0F9000F2E0540F75F014A42413F582BA
:104EEF00E43449F583C083C0829000F3E0540FD0BF
:0D4EFF0082D083126821126909126A0F2205
:1067D6009000BFE0F52A1269C71269F7124E8F12B0
:0567E60069CA0269FA16
:106702009000B6E060031269D69000BFE0F52A124D
:0E67120069F71268DB1268F11269FA0269D3A6
:030000000268A3F0
:0C68A300787FE4F6D8FD75816D02462771
:10428900BB010689828A83E0225002E722BBFE0233
:09429900E32289828A83E4932266
:1042A200BB010CE58229F582E5833AF583E02250D1
:1042B20006E92582F8E622BBFE06E92582F8E2221B
:0D42C200E58229F582E5833AF583E4932235
:1042CF00BB010689828A83F0225002F722BBFE01CE
:0242DF00F322C8
:1042E100BC000BBE0029EF8DF084FFADF022E4CCC1
:1042F100F875F008EF2FFFEE33FEEC33FCEE9DEC8A
:10430100984005FCEE9DFE0FD5F0E9E4CEFD22EDCF
:10431100F8F5F0EE8420D21CFEADF075F008EF2F19
:10432100FFED33FD4007985006D5F0F222C398FD0A
:054331000FD5F0EA22A7
:10433600A3F8E0C5F025F0F0E5821582700215833A
:06434600E0C838F0E82297
:0C434C00A42582F582E5F03583F583227C
:10435800D083D082F8E4937012740193700DA3A3F4
:1043680093F8740193F5828883E473740293686008
:06437800EFA3A3A380DF08
:00000001FF
